:020000040800F2
:10000000E81D0020D5000008DD000008DF00000822
:1000100000000000000000000000000000000000E0
:10002000000000000000000000000000E1000008E7
:100030000000000000000000E3000008A54F0008D9
:1000400000000000E7000008E70000083D3E00084F
:10005000E7000008E700000815160008CD160008A4
:10006000051700086D110008A1110008D51100083E
:10007000E7000008255600081D3E0008E7000008BC
:10008000E7000008E7000008A1080008C108000810
:10009000595500089156000879550008E7000008F6
:1000A0004D1600088D160008F92D0008BD540008F3
:1000B00009550008DD2D0008E7000008E7000008EA
:1000C0000348854600F0DAFB00480047E96C000869
:1000D000E81D00200448804704480047FEE7FEE78B
:1000E000FEE7FEE7FEE7FEE731510008C100000829
:1000F000F0B51FB40646002082B0054640240191A9
:1001000000901BE0019922460F46304600F0F1FABC
:10011000049A059B801A994110D31046194622462D
:1001200000F0D7FA361A8F410197224601200021AC
:10013000009F00F0CEFA38184D4100902046641E12
:100140000028DFDC019B00982946324607B0F0BD4D
:1001500030B5434351435C18010C130C0D465D430D
:100160002C1980B292B20546554351430A0C09043A
:100170004D1962415843010C00044019514130BDF2
:1001800010B5431A934209D28318881803E0401E21
:1001900001785B1E1970521EF9D210BD03460B4345
:1001A0009B0703D009E008C9121F08C0042AFAD22D
:1001B00003E00B780370401C491C521EF9D210BD9D
:1001C000D2B201E00270401C491EFBD270470022EF
:1001D000F6E710B513460A4604461946FFF7F0FF46
:1001E000204610BD421C0178401C0029FBD1801A1A
:1001F000704770B502464A40D50F40004A00ED07EF
:1002000040085208002814D0002A12D0C40DD30D83
:1002100041020120C0055202490A520AE41A091893
:1002200012187D34914201D3641C00E04900002C77
:1002300001DA002070BD0023914201D3891A0343E3
:10024000400849000028F7D100290AD0914202D184
:100250000121C90705E0914201D2012101E00121FC
:10026000C943E005C018401900F067FA70BD0000EE
:10027000F0B507460846584087B0C00F04904800C4
:100280000E46590040084908BC1A884105D2384634
:1002900031461E4617460B4602465800400810439A
:1002A0004CD0300D039040055900400D490D05908C
:1002B000401A0290402872DA18030121000B090548
:1002C0000843019004980092002805D001995242F9
:1002D0000020884100920190029840210A1A019959
:1002E000009800F0F6F905460C466B4607CB00F087
:1002F00011FAC0197141039A0E0D0023D717564009
:100300001A467A40164344D0049A002A2DD0029A05
:10031000012A039A15DC1205C01A914101263605FF
:10032000001C7141D20F059ED207009301920296E4
:100330002A46234600F04FFA07B0F0BD3846314652
:10034000FAE71605224A0F46B218C01AB741012132
:100350000905001C4F4100187F41114618187941CA
:10036000E20F10436D19644113E0E2076D08154375
:100370006408C2071443039A01261205C01A91416A
:100380003605001C7141CE07400830434908C018AB
:1003900051412A46234600F011FACDE7FFE70498C1
:1003A00001224000C117121A00238B4104983146E4
:1003B000C417381AA141EEE730B40124E4076340C2
:1003C00030BC55E730B40124E407614030BC4FE74E
:1003D0000000E0FFF0B51FB488B00B990998002425
:1003E00048400999C00F490049080991C0070B9975
:1003F0000090490049080B9109990898A6460843BE
:100400001CD00B990A98084318D009980124400081
:10041000420D4800410D099824050003000B2043BC
:1004200009900B980003000B20430B9050181C49B7
:100430004018002201901446104605E000200146B5
:100440000DB0F0BD032801DA034600E003239C460B
:10045000C11A0AAE0AE05F0008ADED5B4F00F75B22
:100460007D430027AA187C41491C5B1E6145F2DDD3
:10047000410004AB5A522104120C0A43240C401CC4
:100480000828DFDB019802900099704601910090E6
:10049000059B049A0799069800F09DF9D0E70000A3
:1004A0000DFCFFFFF0B50C465C4085B0E40FE4079F
:1004B00003944C00002664085900944649080246FB
:1004C0000296224321D062460A431ED06200570D95
:1004D0004A000E032303550D012402462C4924052E
:1004E000781B1B0B360B40182343264361460090B4
:1004F0001C46501AB44103D30098401C009002E0FF
:10050000921800985B41002803DA0020014605B0EC
:10051000F0BD0020012109050746864611E064462A
:100520001D46141BB54106D36546521BB3417446A4
:1005300007430C43A646CD074008490828439218B4
:100540005B4105460D43EAD11046184313D060467F
:10055000194650407140084306D06046101AB34116
:1005600006D20122002306E000220123DB0702E07D
:100570000122D2435310009874460105381C614192
:10058000029C039D0019694100F018F9BFE70000C3
:10059000FD030000C217C10F504010B54018CA0734
:1005A0009623002100F0D1F810BD10B5002296234B
:1005B000114600F0CAF810BD0EB5054902910021A0
:1005C00000910A460B46019100F005F903B000BD09
:1005D000330400000EB5054A029200220092134631
:1005E000019200F0F8F803B000BD000033040000F1
:1005F0004A0009030123090B1B051943094B10B5D8
:10060000520D9A4201DA002010BD064B34339A4253
:1006100003DC9A1A00F06DF810BD034951188840A8
:1006200010BD0000FF030000CDFBFFFF4A000903DF
:100630000123090B1B0519430A4B10B5520D9A42B1
:1006400002DA0020014610BD064B34339A4203DC27
:100650009A1A00F04EF810BD034BD21800F039F88A
:1006600010BD0000FF030000CDFBFFFFC20FD2074B
:10067000400040080BD0C10D0723DB01C918400220
:100680000905400A1143C208400711437047002082
:100690000146704770B50446002903D0002020228F
:1006A000012310E0002801D00020C043C046C0460E
:1006B0000DE02546D5408D4205D30D469540641B7F
:1006C0001D46954040191546521E002DF1DC21466D
:1006D00070BD10B5202A04DB0146203A914000206D
:1006E00010BD914020239C1A0346E34019439040DB
:1006F00010BD10B5202A04DB0846203AD040002166
:1007000010BD0B46D340D0402024A21A914008438C
:10071000194610BD10B5202A06DBCB170846203A33
:100720001041C1170B4306E00B461341D040202473
:10073000A21A91400843194610BD002904DA401C52
:10074000490001D140084000704770B40024050CF6
:1007500005D11024000402D1002921D01124050E56
:1007600001D100020834050F01D10001241D850FBD
:1007700001D18000A41C002801DB4000641C00297A
:1007800008D020252E1B0D46F540A14000D00121A8
:100790002943084301061B1B000ADB1D02D500206C
:1007A00070BC7047DB05181880180029F8DA401C67
:1007B0004900F5D170BC40084000704710B5002BCF
:1007C00008DA0024401C614192185B411A4301D1B0
:1007D0004008400010BDF0B51FB482B005460C00C3
:1007E00003D0084606F0BCFA02E006F0B9FA203061
:1007F0000246009021462846FFF76BFF049B059AAE
:1008000004460F4618431143084314D018461043BA
:100810001BD0009840210A1A18460599FFF769FF76
:1008200005460E46009A05990498FFF752FF0843C3
:1008300005D0012004E02046394607B0F0BD002075
:10084000C11705430E432C43374300990E986305A7
:10085000401A7905E40A00220C43FD0A0A3002D549
:1008600000200146E9E70105101969410C9C0D9D26
:1008700000196941FFF7A2FFDFE70000064C0125E0
:10088000064E05E0E36807CC2B430C3C9847103438
:10089000B442F7D3FFF718FC1C9100083C91000804
:1008A00080B50120010301F05DFC012804D103485B
:1008B0000068002800D0804780BDC046DC0E0020C4
:1008C00080B501200103022001F04CFC012804D175
:1008D00002480068002800D0804780BDE00E00205C
:1008E000B0B584B00D46044669464D710A7108984A
:1008F000C8708B70002088720125CD800D80FF208C
:1009000002300881204601F055FC204629462A463F
:1009100001F036FC04B0B0BD80B582B001AA917080
:10092000107000205070104602F03CF902B080BDFB
:1009300080B501F0B7FC80BD80B500F001F880BD46
:10094000F0B5CDB04BAE0024B471FF200230B080C2
:1009500034484B90344D2846314601F039FFB4718C
:1009600001273802B08031484B902846314601F0CB
:100970002FFF08212846224601F0B5FF1021284606
:100980003A4601F0B0FF7D20C00006F07BF928490F
:1009900028A048610320488104F0BEF90A2006F02F
:1009A00071F9641C642CF9D1234881780A9141784B
:1009B0000991C178047946798779C579027A437AB1
:1009C000807A00910194029603970495059206930C
:1009D00007900BAC19A12046099A0A9B06F0ACF9C6
:1009E0002046FFF7FFFB0104114D04D00BA96961FC
:1009F000688104F091F900240A2006F043F9641C90
:100A0000642CF9D118A068610920688104F084F988
:100A100000240A2006F036F9641C642CF9D14DB08C
:100A2000F0BDC046080001000008014010000100B0
:100A3000240200202B2B2B000100002041542B4EC0
:100A4000414D453D312C35333439343135322578FB
:100A500025782578257825782578257825782578AE
:100A600025780D0A0000000041542B455849540DCB
:100A70000A000000B0B582B0044601A900208870C9
:100A800001250D80064801F037FC2846214601F07B
:100A9000B3FC2846294601F06BFC02B0B0BDC0464D
:100AA00000A402407047000080B507480178012289
:100AB0000A43027004F02EFA044801F05DFE044877
:100AC00001F05AFE80BDC0468E0F002008010020B4
:100AD0003001002010B50122012804D0022809D1DC
:100AE0009405064A01E01405034A116001F02CFC4C
:100AF0000348046010BDC046F00E0020F40E002034
:100B000000E100E010B500290CD00023074ADBB259
:100B100004785C40135D401C491E0C06F7D1D84395
:100B2000C0B210BDFF20C0B210BDC0463672000872
:100B300010B50C4800890C490880CF2040003B4C80
:100B4000205A0C49884206D00B49884209D1BC344E
:100B50009520400002E0054C0E34054805F0E4FF06
:100B6000208010BDA815002068150020FA0D002077
:100B700015040000514B00005A4A00007047000065
:100B80000B48052101760B4909680B4A914205D0B3
:100B90000A4A914202D00A4A914204D109490022EC
:100BA0000A800276704700218180074801807047E3
:100BB000240200204C15002055AA000033313032A9
:100BC0004452495322020020DC12002080B5044820
:100BD0000021818101604160816004F003F880BDE3
:100BE000F40100207047000010B5B6200F490C5AE0
:100BF0000F4804800F480068FFF7CCFC0E49FFF750
:100C0000F8FA0E4908602046FFF7CFFC0C49FFF7C1
:100C1000F0FA0C4908600C480068FFF7BBFC0B4970
:100C2000FFF7E7FA0A49086010BDC04640020020FD
:100C30000C02002008020020F902155014020020C6
:100C400000007A44180200201002002000401C46D8
:100C50001C020020F0B587B00546401E81B2022973
:100C600000D9DDE1BA4B1F88BA4C268800B240009B
:100C7000B949095A2180B94A1180B949085AB94974
:100C800008801880B849088006F00EF82288B74816
:100C90000068B24204960295019746D0052E069050
:100CA00009D8E348E349C0467E4436797600B74424
:100CB000100205080B0EE84800210AE0E448E54967
:100CC00007E0E148E14904E0DD48DE4901E0DA48B7
:100CD000DA49E24B19605860052A08D8DC49DD483A
:100CE0007A44127952009744100205080B0EDA4933
:100CF00000200AE0CE49CF4807E0DD49DD4804E0A6
:100D0000D949DA4801E0D649D6480CCBFFF762FB57
:100D100004460E460698FFF74FFC02460B46204657
:100D20003146FFF757FBFFF763FCD3490860BF4D1F
:100D30002860FF200A300390801D05F035FEAC21AD
:100D4000CE4F7852CE4908604988AA22B95228600D
:100D5000B5480288CB4D2E68049CA24248D0052C91
:100D600009D8B348B349C0467C4424796400A744F9
:100D7000100205080B0EB84800210AE0B448B54936
:100D800007E0B148B14904E0AD48AE4901E0AA48E6
:100D9000AA49B24B19605860052A08D8AC49AD4839
:100DA0007A44127952009744100205080B0EAA49A2
:100DB00000200AE09E499F4807E0AD49AD4804E0A5
:100DC000A949AA4801E0A649A6480CCBFFF702FBB7
:100DD00004460F463046FFF7EFFB02460B4620461F
:100DE0003946FFF7F7FAFFF703FC0646A34F049CCA
:100DF000A14806602E60039805F0D6FDA821785220
:100E0000D94908604988A622B952286001204002C9
:100E10000690385A002872D000259B4E09E00F46F4
:100E200001C6E8B204F09EF80698385A6D1C854257
:100E300065D239467C4807883068A742EFD0052C38
:100E400005901FD8A10003A253587A49784A834CD1
:100E50009F46C046910E00086D0E0008730E0008F4
:100E6000790E00087F0E00088D0E000800217A4AD6
:100E70000EE07849764A0BE07449734A08E07149FC
:100E80006F4A05E00021744A744C01E06B496A4ADC
:100E900006C4083C052F11D8B80002A10A586D48B5
:100EA0006B499746D90E0008BD0E0008C30E000816
:100EB000C90E0008CF0E0008D50E000800206649B4
:100EC0000AE05C485A4907E06A48694904E0674813
:100ED000654901E0634862490CCCFFF77BFA0446A0
:100EE0000F460598FFF768FB02460B462046394639
:100EF000FFF770FAFFF77CFB604F049C90E74948CE
:100F000000880199814200D181E04B1E032B07D854
:100F10005E495F4A7B441B795B009F4409010407DB
:100F20004D49002204E05D495D4A01E059495A4AB1
:100F30004A4B1A605960401E0026032818D8594FA2
:100F40003446C0467844007940008744191114178C
:100F5000B2000020841200202A72000886120020AD
:100F600030720008B4000020B0000020D012002031
:100F7000394F344604E04E4F4E4C01E04A4F4B4C43
:100F800003F0FEFA03F0A4FA4B4D03CD083DFFF742
:100F900021FB02460B4620463946FFF71BFA024664
:100FA0000B462E4903C9FFF715FAFFF73FFB07462B
:100FB0000C46424A3346FFF79BF8414A1060F34320
:100FC000404AFFF7C5F8C01928603F4A10606141E8
:100FD00069603E4C611D092201273B4600F07CF808
:100FE00037480068052221463B4600F075F803F0BB
:100FF0003BFD03F087FA00F0E1FB701C042E06466F
:10100000F9D3334800210180324801601B4F029818
:10101000554908800398273005F086FDC021785295
:1010200007B0F0BDB200002084120020D0120020D2
:1010300051B8AE3FB81E85EB5F34DE3F1188B2CAAF
:101040009AA92B40BD9AA9BB19513C40905F07CE8D
:10105000AAAA3040ABAAAAAA0000F03FB81200200A
:1010600079F30040A8FCE02F4082B23F6D3480B796
:10107000C514A23FE6736788601500204002002077
:1010800068150020D81200209C1100204D62503FAE
:10109000FCA9F1D2578EEA3F1A578E1A14FF9C3FD3
:1010A00058A1B54700408F40AE47F33F48E17A145E
:1010B00048A841402F0735E79012002000CA9A3B0C
:1010C00098150020003665C49C150020F40100200E
:1010D00074120020B0120020F0B581B014460D4605
:1010E00006460027002B03D0F943002C03D115E05E
:1010F0000121002C12D0002B01D06019451E009157
:101100000A213046FFF7C6FAF621414389192970B2
:1011100000996D187F1CA7420646F1D301B0F0BDBF
:10112000B0B51048018900290DD00F4A521E002386
:10113000C488651CC580515C05692955521E5B1C1D
:1011400001898B42F4D382888B1C934202D90021FF
:101150008180B0BD4B080381511A81800188C91874
:101160000180B0BD240200206815002080B5002059
:1011700001F064FA042804D1DC480068002809D191
:1011800009E0002001F05AFA022804D1D74840684B
:10119000002800D08047002001F074F980BDC046CF
:1011A00080B5012001F04AFA042804D1CF488068B4
:1011B000002809D109E0012001F040FA022804D1F9
:1011C000CA48C068002800D08047012001F05AF9C1
:1011D00080BDC04680B5022001F030FA042804D159
:1011E000C2480069002809D109E0022001F026FA6E
:1011F000022804D1BD484069002800D08047032060
:1012000001F01CFA042804D1B8488069002809D1EB
:1012100009E0032001F012FA022804D1B348C069A2
:10122000002800D08047022001F02CF9032001F0B3
:1012300029F980BD10B5A34C2078FD210140217013
:101240009E4801F099FA2078FE210140217000208B
:10125000152100F063F8A01C784C20612078400133
:101260000549421821460C31204601F011F920466B
:1012700001F078FA10BDC04600900240F0B581B090
:1012800015460C4602281FD0012843D101273846B5
:10129000394600F059FF0220192100F03FF8812063
:1012A0004000354E708431460C3100224A75F5827B
:1012B000B782B2701849F16034613080304601F075
:1012C000E1F9002821D0FEE702200127394600F08D
:1012D0003BFF03201A2100F021F881204000274E17
:1012E000708430460C3000214175F582B782B170B0
:1012F00009482C30F0603461FF20043030803046E3
:1013000001F0C0F9002800D0FEE70221012230469A
:1013100001F0A8F901B0F0BD9C28014080B582B071
:1013200001AA11705070012000025080104601F097
:1013300095F802B080BD000010B50446012801D028
:101340000E4800E00C4801F00DFA012C00D00224F8
:10135000204600F0B3FF10BD10B50446012801D0AF
:10136000064800E0044801F007FA012C00D00224EE
:10137000204600F0B1FF10BDB8000020E0000020C2
:10138000F0B59BB00190002415212046FFF7C6FF61
:101390002A4F384601F0F0F9BC700125680202902E
:1013A00038804848801C4649254AF96038617A618E
:1013B0002448386203AE384601F064F9002800D0B2
:1013C000FEE72C36204F032078703C701F480168E0
:1013D000232048430199FFF75DF9401E80B2FFF7D3
:1013E00049FB1B492846FFF775FB03A88474048258
:1013F0000299F1807471B5701390164812901649D5
:101400001191164904910397154A0592034620331A
:101410000693144B08930B91791C0A910C920D9032
:1014200010203071348011A801F02CF9002800D070
:10143000FEE7024801F096F91BB0F0BD080100205C
:1014400001000001010100015801002010000020EE
:10145000A90A0008600100200104000208A502405A
:10146000010001001000000210B5002414212046E4
:10147000FFF754FF1148847001210A0202804A02DA
:1014800042840F4A818203460C33597581214900F9
:101490000C4B5918C16002610B49595CC18201F0C3
:1014A000F1F8002800D0FEE7044C0221012220467A
:1014B00001F0D8F8204601F055F910BD30010020A8
:1014C000003801408E0F00200302000010B5C30059
:1014D000064CE150E1184A60032805D840B280006C
:1014E00003A108580649086010BDC0461C12002020
:1014F00000020000000400000008000000080000D6
:1015000000E100E0F0B583B034480468344E7D203B
:101510000190C700776060080290F0603461642534
:1015200020462946FFF7B6F830600A206043294676
:10153000FFF7B0F80546B0602A48844202D8019807
:10154000800030603068B84205D3052060436421D4
:10155000FFF7A0F8706070688542029A02D8801880
:101560004008B060B068824202D800194008F060BC
:10157000012044021C4D052028531C4A1070384697
:10158000D83805F0D1FA285B002825D022463B4602
:1015900000200646174DF1B217464A00144CA352DC
:1015A00089000F4A5158114A11602B806980518877
:1015B000A9800722504303214902401880B21C46EB
:1015C0000223294605F062FA23463A460648C15BE3
:1015D000761CF0B28142DED803B0F0BDD0120020FC
:1015E0009C1100204FC3000040020020681500201D
:1015F000EC1100206015002010B5054C0521204697
:1016000000F0A5F820210122204601F06CF910BD60
:101610004008014080B5012001F0B8F8012807D149
:10162000012001F0AFF844480068002800D080474E
:10163000022001F0ABF8012807D1022001F0A2F846
:101640003D484068002800D0804780BDB0B50125E6
:10165000AC02204601F09AF8012807D1204601F09B
:1016600091F83548806A002800D08047EC02204677
:1016700001F08CF8012807D1204601F083F82E48AC
:10168000C06A002800D08047B0BDC046B0B5012573
:101690002C03204601F07AF8012808D12648006B77
:1016A000002800D08047204601F06CF8B0BD6C03E4
:1016B000204601F06BF8012807D1204601F062F8BE
:1016C0001D48406B002800D08047B0BD80B5042085
:1016D00001F05CF8012807D1042001F053F8164806
:1016E0008068002800D08047082001F04FF80128CA
:1016F00007D1082001F046F80F48C068002800D044
:10170000804780BD70B50C4D1035042603E02D1DBB
:10171000761C082E0FD00120B04084B2204601F084
:1017200035F80128F3D1204601F02CF8286800286C
:10173000EDD08047EBE770BD3C12002001228A40CB
:101740004168914341604169114341617047B0B5BF
:1017500001231A468A404468144344604469944310
:101760004461490003248C40056AA54305628B400F
:10177000016A19430162016991430161B0BD01220F
:101780008A40C1689143C16081681143816070479C
:1017900080B50648008840000549085A03F0DCFA85
:1017A0000448054905F082FA80BDC0464415002072
:1017B0005E740008000C00407D3D0008F0B585B067
:1017C0002D4A1078401CC1B2042900D900201070A5
:1017D00001212A4C04E01070029A511C032A47D8B8
:1017E0000291C0B20E2141430920000201910D185F
:1017F000072602272846214632463B4605F046F991
:1018000003A9284632463B4602F050FD0020215CE9
:1018100003AA125C8A4220D1411C05280846F6D949
:101820004920800101990D180726022728462146E4
:1018300032463B4605F02AF903A9284632463B4684
:1018400002F034FD0020215C03AA125C8A4204D11C
:10185000411C05280846F6D907E0074A1078401CC5
:10186000C1B20429B7D90020B5E7002005B0F0BD0A
:10187000012005B0F0BDC046E0040020EC0D0020C2
:10188000F0B583B04D4F788806283FD8784400796A
:1018900040008744033E6587878787004848017872
:1018A000FE220A40027010200290009001240321C1
:1018B00001910026072320463246FFF711F8112038
:1018C000009002252846019932462B46FFF708F87A
:1018D00002983881FE802046FFF72AF83A7A394686
:1018E00024312046FFF7CAFC4F20800039183A7A8D
:1018F0002846FFF7C3FC2046FFF71EFD2846FFF7EA
:101900001BFD7C8005208001B8804BE000207880A2
:1019100048E001242046FFF71FFD0220FFF71CFDD1
:101920000020F8613862E1037F22D243403203464F
:10193000BC185F25AD0065592D0A6D18ADB2281889
:10194000646E240A6418A4B2E318121DF0D10321B6
:10195000798000091909F9613862F960386121E07C
:1019600001242046FFF7F8FC0220FFF7F5FC0020D9
:10197000F8613862E1037F22D2430346BC186F2529
:10198000AD0065592D0A6D18ADB22818A42564590B
:10199000240A6418A4B2E318121DEFD140095909B2
:1019A000F96138627888002804D0B88803F07EFA9C
:1019B00003B0F0BD03F0B6FA03B0F0BDF0120020A2
:1019C0002002002070B5684904220A818A88032A0F
:1019D00006D86648002202808A800320087670BDFF
:1019E00000220A76614A01231380CA88551CCD80E3
:1019F0000B699E5C844CE670961CCE80ADB25D5D3A
:101A0000A570D51CCD80B6B29E5D6670121DCA80D1
:101A1000A9B2595C21702168016070BD70B552494E
:101A200002220A818A88012A06D8504800220280B0
:101A30008A800320087670BD00220A764B4A012373
:101A40001380CA88531CCB800C69A55CF04E75705E
:101A5000921CCA8099B2615C31703188018070BD7E
:101A6000F0B583B00446E748042505818588032D39
:101A700009D83E4D00262E808680032505769042AB
:101A800025D903B0F0BD00250576384D01262E80FE
:101A9000C5880291019323466C1CC4800669715D60
:101AA000594FF970A91CC180A4B2345DBC70EC1C04
:101AB000C48089B2715C7970291DC180A0B21C46B6
:101AC000019B0299305C387038689042D9D89842AE
:101AD000D7D322688242D4D024480122028008460B
:101AE00004F062FF206003B0F0BDC046F0B583B0E3
:101AF00002910446C348022505818588012D09D835
:101B00001A4E0025358085800326067695421CD91D
:101B100003B0F0BD00250576144D01262E80C58842
:101B20006E1CC68001931346076922467C5DB84946
:101B30004C70AC1CC4801446B0B2385C1A46019B91
:101B4000B34908700D889542E2D89D42E0D32088C1
:101B5000A842DDD0054801210180029804F0E4FF8D
:101B6000208003B0F0BDC04624020020DC1200201B
:101B7000F0B583B0FF2434340125E903204602F098
:101B8000E5FBC221354E70527D20C100E01C02F001
:101B9000DDFBC4217052E80200210190029102F0A5
:101BA000D5FB16490880002826D0154F154C029DFC
:101BB00007E03880A41CBF1C6D1C104800888542BB
:101BC0001AD205221046684301990818801C80B279
:101BD00002230D490E4602F069FB30463679042196
:101BE000FEF790FF86420298E3D100200649087173
:101BF000488820800888DCE703B0F0BD96110020FB
:101C000068000020200000206015002080B5002022
:101C100000F00EFD0249401A801E024A885480BD21
:101C20008E0F00200202000070B50D204001E34934
:101C300008180B4C206000250A4E715D0320684394
:101C40000522D201801880B202F080FB2168088052
:101C5000881E20606D1C302DEFD170BD4002002029
:101C6000E0010020F87300087047704770470000DB
:101C700070B5094C08340025084E052068435521ED
:101C80000901401880B2216802F078F901C60C34CD
:101C90006D1C102DF1D170BD38730008A00100201B
:101CA000F0B581B0C04DA888022800D2A7E0564BFD
:101CB000C84C06E001F0D0FAA8880128524B00D8A1
:101CC0009DE002272F812888FF260146B1434F4A15
:101CD0008918090A06294CD87944097949008F44A2
:101CE000034854115748330002F066F95BE01030A6
:101CF000C006800E4C49085A2080FFF711FAA888C8
:101D0000012850D92F8128880F2201469143424A49
:101D10009142ECD0414A9142E9D083221202914291
:101D200005D140003E4940183E49405AE0E73F494E
:101D3000884238D80020DFE700202080FFF7F0F944
:101D4000A8880128304B2ED92F8128880146B1431D
:101D50001A46203A92B29142EED1984223D84000DE
:101D60002C49401880B202222146134602F09EFA06
:101D7000E4E70F21090301400D22120391420AD02A
:101D80000720400381420CD121E002F0A9F90AE0CA
:101D900002F03AFA07E0DF210902884201D1244823
:101DA00000E0002020802889002800D182E701215E
:101DB000EA88531CEB808BB280B2C01A205C2B697E
:101DC00098542889491C8AB29042F1D272E77C4823
:101DD00000887C49884208D07B4988420BD1012089
:101DE0000003F02102F056F807E0DD20C0015A217F
:101DF00002F050F801E0042028760020A88001B00D
:101E0000F0BDC04624020020208600000080FFFFB5
:101E10006815002080FDFFFF208300001083000074
:101E20003474000800FAFEFFA8150020308300007B
:101E30005041000070B50A48041D0025094E0320DA
:101E4000684301218902401880B2218802F07EFA9D
:101E50003080A41DB61C6D1C702DF0D170BDC04625
:101E600076740008FA0D0020F0B581B04E4D0026C2
:101E70002E814E4801684E4A914200D1066001F021
:101E800001FA002801D001B0F0BD4A4F05E000F092
:101E9000EDFF01F0F7F90028F5D1474806802988C1
:101EA000FF240A46A243212080028242F1D0412031
:101EB00040028242EBD00120C3039A4222D1A8887B
:101EC0000228E6D328880146A1433A460A329142C5
:101ED0000AD10C202881A8880B2833D910210C2284
:101EE000364804F081FD05E0C01980B2692801D8A8
:101EF00004F05AFC01F0C6F90028CAD1A8880128CC
:101F0000E0D8C6E70F22120311400D2212039142BE
:101F10001BD1CF2044002948001902F01FFE2B4896
:101F200000880028B5D02548005B2949884203D0A5
:101F30001F498842ADD11AE0264908800D2004F0DF
:101F4000F3FDA6E703202876A3E707225203914278
:101F50000AD11B4909881B4A91421DD01A4A914255
:101F600002D10003F0211AE00420287619E01A4873
:101F700018490880194908800D2004F0D5FD04F0A7
:101F800093FE00F00BFCBFF34F8F1548154901601D
:101F9000BFF34F8F00BFFDE7DD20C0015A2104F0E1
:101FA000B7FBAE8001B0F0BD240200204C1500202C
:101FB00055AA0000F67F0000220200204002002007
:101FC000880F0020464D000054430000DC12002022
:101FD00066BB00006815002055AAFFFFF40D002025
:101FE0000CED00E00400FA05F0B583B001AC00256B
:101FF000A57181204000A080022001904B4E304608
:10200000214600F0E5FBA57101273802A0800C48AD
:1020100001903046214600F0DBFB304639462A4627
:1020200000F061FCA571FF200230A08042480570DD
:102030000197403E3046214600F0CAFB03B0F0BD98
:1020400001000100F0B581B0384C0221204600F0BB
:1020500043FC0546364801788D4206D13548018853
:10206000491C8AB28A4203D003E00570314800213E
:10207000018030480088022855D32F49087801286C
:1020800011D12E4F387801280DD10121002620468C
:10209000324600F028FC642004F0F4FD264928486C
:1020A00006600E703E70087801281DD000283AD1D5
:1020B000012D33D123480078002834D1204E3068D8
:1020C000401C306032282ED3012520460C4629467C
:1020D0002A4600F008FC642004F0D4FD00203060A3
:1020E0002570164908701CE0012D17D1154800789D
:1020F000002818D1124F3868401C3860322812D39B
:102100000125002620460C462946324600F0EBFB0E
:10211000642004F0B7FD3E60267002E00848002508
:1021200005600848057001B0F0BDC0464008014098
:102130009E1200209C1200209A120020981200206B
:10214000A01200209F120020054A002903D0116828
:102150000143116070471168814311607047C046A8
:102160008C280140054A012800D02C321068022931
:1021700001D0012070478007C00F704798280140A8
:102180000B4B012A05D101280AD1186808431860B1
:102190007047C943012807D1186808401860704784
:1021A000D86A0843D8627047D86A0840D862704736
:1021B000A028014070B50C46064601252804294692
:1021C00001F010FE002C62D0022E2DD0012E5ED127
:1021D0000121480201F006FE3048C169304A0A4038
:1021E000C26121788900C2690A436178C90211433A
:1021F000C161E178A27852010A430262A1798902A1
:10220000227A52020A43617A09021143E2791201E9
:102210000A43217911434162617981620168022296
:102220000A430260002070BD0125A802294601F082
:10223000D9FD1A48816C1A4A0A40826421788900C3
:10224000826C0A436178C90211438164E178A27803
:1022500052010A43C264A1798902227A52020A43D6
:10226000617A09021143E27912010A43217911438B
:10227000016561794165016804220A430260816851
:10228000A27A012A05D1AA041143816000252846BB
:1022900070BDAA0491438160002070BD8828014070
:1022A000C3C7FFFF401E414241418802012189020C
:1022B0000F4A13688B4318181060704701214A03B6
:1022C0000B49012803D10868104308607047C86AA9
:1022D0001043C8627047C0460549064A012803D129
:1022E0000868104008607047C86A1040C8627047AC
:1022F000A4280140FFDFFFFF70B50D46044601260C
:102300007002314601F052FD2878401E411E88417E
:10231000400021680222914308182060A878401EDE
:10232000411E88412168B143081820606878401E2A
:102330004142414188002321C900625804239A4345
:102340001018605070BD00000849002804D0012812
:1023500007D0022804D070470868012202430A60AF
:1023600010310868012202430A6070470CA5024040
:1023700000280FD002281FD0012836D13648012965
:1023800026D1416801220A434260016802220A43C1
:1023900002607047304801291FD141680122114372
:1023A000416041691143416101680222914301602A
:1023B00001691143016170472748012916D141691C
:1023C00001220A434261016902220A430261704705
:1023D000016802229143016070470221C9430268EB
:1023E0000A40026002690A400261704701690222E4
:1023F000914301617047C046002806D0022808D0EA
:10240000012805D10448016070470348016001615B
:10241000704701480161704700A5024000280FD0B5
:10242000022807D0012816D10B48016801229143E8
:1024300001607047084801690122914301617047BA
:102440000120C243044801681140016001699142C2
:1024500000D3891C0161704708A5024010B50446ED
:102460000120014601F0A2FCE078C001A1788901B9
:102470000143207808436178014A8854002010BD48
:1024800000A00240014908707047C0461F8002400A
:10249000F0B583B0044608681060486810618F7D0D
:1024A0003802C019D08001252B46BB40487D10283A
:1024B0000190029505D1088B58439080488B434387
:1024C00000E0938093820B890420165E1420155E31
:1024D000C87D052845D80094029C2404BC402414DF
:1024E0005C43E7177C40E71B5E435D43784400791B
:1024F00040008744020B1A2902024A4807409760AD
:10250000488946437342D360454327E04448074027
:10251000704203039B08FB18029CE4071B1993609D
:10252000D06048896843454219E03D4807406D4204
:10253000280380083818029B9B07C01890604889C0
:1025400070434042D0600AE035480740B002381A74
:1025500003239B07034393607042D0606D429561F3
:10256000009C4889D083D082002090836078042822
:1025700029D002280DD001284FD10198C007000FA3
:102580009083D08B28490840D083D08A0840D082DD
:1025900043E0087D0102019BDB071B0F5918203126
:1025A0009183D18B204B1940D1834002D18B0143C1
:1025B0001E4C2143D183D18A1940D182D18A014353
:1025C0002143D18229E0487C8000019BDB071B0F5F
:1025D0000343087C400018438B7C034310201843BE
:1025E0009083C8689061D08B0F4B1840D083D08AFD
:1025F0001840D082087D10280FD0D18B4302194398
:102600000A4C2143D183D18A19432143D18200024C
:10261000918B0143202008439083002003B0F0BD3C
:10262000FF030000FF3F0000FF7900000080FFFF74
:10263000400101494058704710900240400148490C
:102640004018818B490709D5C18A054A0A40C08BC9
:102650004008C0B2824201D804207047022070476F
:10266000FF01000010B500784001054BC45A012A53
:1026700002D00C40C45210BD0C43C45210BDC04621
:102680001C900240F0B581B0054601242046214649
:1026900001F08CFB31490868002846D428788876F8
:1026A000C877887780220A60697804293FD1A868B2
:1026B00000284BD06868002848D00094E8780028AB
:1026C00015D000273C463E46A868C1194889002815
:1026D0003FD0088900283ED0686802192846FFF7D5
:1026E000D7FE1C372034761CE8788642ECD3686825
:1026F00001682A7852011A4BD150D11882888A80F9
:10270000C288CA8082688A60C268CA6002690A6137
:10271000828A8A82C28ACA8282698A6100248C8300
:10272000828B8A83C08BC88310E002240EE0E98A82
:1027300000290BD0A98A002908D029460C31400174
:10274000074A82182846FFF7A3FE0024204601B05E
:10275000F0BD009CFAE7009CF8E7C046008002400C
:10276000009002400178034A11708078012800D15E
:10277000917070471B8002400078014908707047D3
:102780001A800240044908607047C046024909683F
:102790000840411E884170471404014070B50B4E3B
:1027A00030680424204330600121204601F028FBDA
:1027B00000252046294601F023FB8020294601F010
:1027C000F5FA3068A043306070BDC0462410024066
:1027D000F0B583B00C46054680200121029101F03E
:1027E000E5FA2688002E75D000210A460B46019690
:1027F00017E0A868B843A860E868B843E8600F200D
:1028000090402E6886432E60A07990402E68064343
:102810002E60019E5B1C3046D840891C121D00288A
:1028200058D0029F9F403742F4D0A678022E16D08F
:10283000012E08D0002E23D16E68BE436E606E69F3
:102840003E436E612BE06E683E436E602E69BE4370
:102850002E6103268E40286AB04328620AE0686829
:1028600038436860286938432861032088402E6A0D
:1028700086432E62E07888402E6A06432E620EE080
:102880006868B84368606869B8436861A869B84314
:10289000A861A868B843A860E868B843E8606079B0
:1028A000002802D0A869384301E0A869B843A861AC
:1028B0002679022E08D0012E9BD1E868B843E86043
:1028C000A8683843A8609AE7A868B843A860E86891
:1028D000384393E703B0F0BD406A0840411E884189
:1028E000704741637047002A02D02C228150704704
:1028F000302281507047000070B50022002934D08A
:10290000814232D242080243900810430209024336
:10291000100A1043020C0243D0434308144A1340E8
:10292000C31A14489C08034004401B191C091D19B4
:10293000114B1D40114C65432D0E4E080E43B1083E
:1029400031430E090E43310A31430E0C0E43F1435D
:102950004E081640891B8A08014002408818010968
:10296000401818406043000E421BD0B270BDC046F4
:1029700055555555333333330F0F0F0F01010101F7
:1029800004494868C00702D1002008607047012050
:102990007047C046103000400348007803490A6879
:1029A000101808607047C04614000020A4150020CD
:1029B000016880220A4302607047000080B5002150
:1029C000016041608160C16001610122254B984234
:1029D00003D0D00701F0F8F980BD900701F0F4F9B9
:1029E00080BDC0460268802313430360491E4A42EB
:1029F0004A419101026840239A435118016070478F
:102A000070B50D46044601261648844201D0F007F1
:102A100000E0B007314601F0D7F92068B0432060EC
:102A20002878411E884140002168022291430818FD
:102A30002060E878411E884180002168042291438B
:102A40000818206060687F2188436060A87881084A
:102A500011406A78636813430007400E1843084327
:102A6000606070BD000C00408160016881220A43F3
:102A700002607047F0B583B00E4604460125A803F6
:102A8000324F39688143226812030240501838607F
:102A900000BF2078C0070AD001A902208871002059
:102AA00088700D80280288801948FFF791FE206801
:102AB000032108403A688A431118396000BF711C2D
:102AC0003A681207920F904202D0491EF8D11CE0DA
:102AD00000BF3868F021884361680901014339600B
:102AE00000BF072001023A688A43A1680902114326
:102AF000396000BFC00239688143E068C002084302
:102B0000386000BF02F066FA0025284603B0F0BD29
:102B1000400801400D4800684005400F042801D3DB
:102B2000C11E00E000210A480068C8407047C04646
:102B3000064800688004400F042801D3C11E00E04D
:102B4000002103480068C8407047C0460410024096
:102B50001000002070B50546012420070F4E316893
:102B600001433160E006316801433160204601F0E5
:102B7000F7F87068012D09D120437060084871682A
:102B8000890708D4401CFAD3204670BDA04370606A
:102B90000024204670BD002070BDC0461C100240BD
:102BA0000000FFFFB0B5044601252804294601F0C6
:102BB00019F9002C28D0154801682278042A02D17E
:102BC000082291430AE0FF2304339943016001681E
:102BD0000A4361780B021343082119430160A2786C
:102BE0000168042A02D1402291430BE023231B01F8
:102BF00099430160110102680A43E1784B021343D3
:102C000040211943016000252846B0BD1C28014021
:102C1000F0B581B001221649164B1C4602E0641C37
:102C2000012E07D0664266410F8820253D40F6D030
:102C30001646F4E70124002D17D002E05B1C012E9C
:102C400007D05E425E410F8808253D40F6D016460B
:102C5000F4E7002D09D00A8882430A800024800707
:102C600003D501204002FFF78DFD204601B0F0BDE5
:102C7000042800400100FFFF574A4A4002617047A4
:102C8000002A03D0C2680A43C2607047524A5140CA
:102C9000C2680A40C2607047B0B50D46044613488A
:102CA000844204D00120014601F08EF803E00121A6
:102CB000C80201F097F820686988E1622988A1625A
:102CC00069794A1E9141C9013F22120190432A7934
:102CD0000243E888104380229043401820606069D6
:102CE00001210143616100202061B0BD002C014041
:102CF000016801220A430260704700000168024A2D
:102D00000A4002607047C046FEFF000002460020F5
:102D1000022909D004290ED15168C9070BD0516985
:102D2000C90708D0012070475168890703D5516948
:102D3000890600D501207047F0B581B00D460446E4
:102D400024480121844205D0480401F03DF8FFF7F2
:102D5000E1FE04E0880301F045F8FFF7E9FE07090A
:102D600000952D6838462946FDF794FC064628460E
:102D70007043381A0001690840182946FDF78AFC9B
:102D80000F2800D9761C1449E26FD20706D04A1EDC
:102D900009041146F8D1032001B0F0BDE26880219A
:102DA0000A43E260F2B22260320AD2B262600F22BB
:102DB0001040C022A050009B9888DA8802431889EE
:102DC0001043E2680243E260E0688843E06000206C
:102DD00001B0F0BD00380140FFFF000080B504489D
:102DE0000068002800D080470248FFF7E1FD80BD61
:102DF000C4120020000C004080B504480068002880
:102E000000D080470248FFF7D3FD80BDC8120020E4
:102E1000200C004010B50F4801880F4A11800F4C5C
:102E20002288028048000E49085AC0090D4B1880BC
:102E30005000085A01F0D0FB0B480178DF220A400D
:102E40000270080702D50120208010BD4448008A86
:102E5000208010BD44150020461500204815002094
:102E60005E7400088C15002092110020F0B581B02E
:102E7000F54CA08802286BD3FB20C701354E05E036
:102E800000F072F82F46A088012861D93D462788B6
:102E9000B742F5D300202081FDF772FE3046703036
:102EA00086B200F0EFF9B74226D20028294E2F460D
:102EB000F34CE8D1208831466F3189B28842E2D89C
:102EC000391870318AB26F2A3FD85000244B181835
:102ED00006235343234DEA5A03264E430121890218
:102EE00071181C4E89B2EB185B88FEF7FFFD00F0ED
:102EF000C9F90028DED0C6E70028164E2F46EA4C56
:102F0000C1D120883146EF3189B28842BBD8C1197E
:102F10000804000E19D1FF2081438AB290000E4BA5
:102F200018180C2353430D4DEA5805264E435521DE
:102F300009017118074E89B2EB185B68FEF790FD26
:102F400000F0A0F90028DCD09DE7022020769AE767
:102F500001B0F0BD10820000A0010020387300080D
:102F6000FA0D002076740008F0B581B0CE4EB0881E
:102F7000022800D272E03B4FEE4C964D0220308189
:102F80003088C1190F291FD87944097949008F4425
:102F900007282C28282828282828282828323D4B8C
:102FA0002046FEF70FFD20683049884202D03049A4
:102FB000884201D12A48206020682949884245D1A9
:102FC0000020DB49088041E02749884209D103F00D
:102FD0006BFE03F0C5FD002003F01CFB03F065FE53
:102FE00034E0000A822831D938E0284601F0B6FDE5
:102FF000FEF73CFE2AE0284601F0B0FDFEF735FE64
:10300000CF2040002988914A11521FE0F088411CCE
:10301000F1803269135C6B70801CF08088B2105CA8
:103020002870FEF721FE11E0F088411CF180326922
:10303000135C6B70801CF08088B2105C2870CF200D
:1030400040002988814A1152FDF772FD00F01AF9FB
:10305000002803D1B088012800D98FE701B0F0BD66
:1030600044524953007EFFFF0680000052414953FD
:1030700033313032F0B581B08B4C00252576206994
:103080004178C91E0D293AD87944097949008F44FD
:103090000636362236333636363636363638C17848
:1030A0008278120251182180427903791B029A1802
:1030B000A28093B2332B31D209B252006281A28036
:1030C00082700320E0806089001D608100297CD42B
:1030D00002F0D2FC24E0C1788078072262813C4A69
:1030E0006260000240182080411C618000B200280C
:1030F00068D402F0D1FD13E00078002810D101203F
:103100000DE0C1788278120251182180427903794A
:103110001B029A18A28093B2332B47D30420207647
:10312000207E00280BD021694A78802313434B70FE
:10313000216901228A702169C87005206081206997
:10314000017800292ED06189002929D00091FE3113
:10315000CAB23F4F3F4B04E06E1C95420F463546C6
:103160000BD0415D7940082702E031467F1EF3D045
:103170004E08C907F9D05E40F7E7164A118051782A
:10318000009BC154206961890818401E11780170A4
:103190006089421C62816069216992B2FCF7F0FF8C
:1031A00001B0F0BD0020608101B0F0BD5300A380EC
:1031B00051186180102141700720E0806081605FBC
:1031C000002896D5FEF750FEAAE7FEF769FDA7E7AF
:1031D0000200040068150020F0B581B032490020DB
:1031E00048818B89052B08D309690A78002A06D003
:1031F000A224164D2C5B944201D001B0F0BD5818AA
:10320000821E12780092401E0278FD33DBB2002548
:103210000F4F104C04E06E1C9D42074635460BD004
:10322000485D7840082702E030467F1EF3D046080C
:10323000C007F9D06640F7E71102009A8918091A09
:103240004842484101B0F0BD240200204002002065
:10325000FFFF000001A00000134881880289931C31
:103260008B4203D9002181800120704753080381DC
:10327000891A81800188C918018000207047C046E2
:103280002402002008490A898B88012093420AD32E
:103290009B1A8B809BB2022B05D3500808810A88A9
:1032A00010180880002070472402002070B51F48C5
:1032B00000881F490A8812180A8092B2520A0F2AFF
:1032C00008D31C4A002313600B801B490A7808238B
:1032D00013430B7019490A78130714D5184B1C882F
:1032E00024181C80A5B2174C2688B5420BD3402564
:1032F000258000241C8080231A430A70124A137808
:10330000BF241C401470114A136818181060000B79
:10331000E1280AD3002010604878FE2202404A705B
:1033200008782522024080320A7070BD8C1500207A
:10333000220200204C1500202002002092110020C3
:103340008A0F00208C0F002058150020E404002074
:1033500080B50D480168491C01600A2905D3002188
:1033600001600A482021FFF7BCFA09480168491C9E
:1033700001600848814202D3074801210170FEF72D
:1033800061FE02F0C5F980BDC012002000080140B6
:1033900050150020411901009812002010B500209E
:1033A000A04980220B4600241C70521E0833002ABC
:1033B000F9D1491C401C0828F3D110BDF0B583B0E9
:1033C0000292994222D20A460299091A0191C40036
:1033D000944D29190091114604E0521C491CCCB2AD
:1033E0009C4213D2029CA042F7D2D408009D2F1910
:1033F00007240C400125A540EC43019D3E78264062
:103400003E706D1E0837002DF8D1E6E703B0F0BD21
:10341000F0B583B00292994222D20A460299091A63
:103420000191C400EA4D29190091114604E0521C93
:10343000491CCCB29C4213D2029CA042F7D2D408C1
:10344000009D2F1907240C400125A540EC43019D48
:103450003E7826403E706D1E0837002DF8D1E6E715
:1034600003B0F0BDF0B583B00292994221D20A4672
:103470000299091A0191C400D54D291900911146EC
:1034800004E0521C491CCCB29C4212D2029CA042C5
:10349000F7D2D408009D2F1907250D400124AC4018
:1034A000019D3E7826433E706D1E0837002DF8D1F1
:1034B000E7E703B0F0BDC046F0B583B001AD00242E
:1034C000AC71012000900702AF8052480190524E2B
:1034D00030462946FFF77CF9AC71AF804F48019028
:1034E000304640302946FFF773F9AC71AF804C4845
:1034F000019030462946FFF76BF9402530462946B2
:103500002246FFF7F0F9C827384603F0BBFB3046E8
:103510002946009AFFF7E7F9AE20214600F052FB5A
:103520000220214600F04EFB1020214600F04AFB0D
:103530002846214600F046FBB020214600F042FB21
:103540008120214600F03EFBCF20214600F03AFBCF
:10355000A120214600F036FBA620214600F032FBD8
:10356000A820214600F02EFB3F20214600F02AFB38
:10357000AD20214600F026FB8B20214600F022FBE7
:103580003320214600F01EFB3846214600F01AFB8E
:10359000D320214600F016FB2046214600F012FB06
:1035A000D520214600F00EFB80263046214600F053
:1035B00009FBD920214600F005FB1F20214600F021
:1035C00001FBDA20214600F0FDFA1220214600F02E
:1035D000F9FADB20214600F0F5FA2846214600F0F2
:1035E000F1FAFC480146324600230B700831521EA6
:1035F000FAD1401C641C082CF4D10920C101F44804
:10360000FCF7E5FD00F010F8AF20002100F0DAFA39
:1036100003B0F0BD100002014008014001000201AA
:1036200040000101E8040020F0B585B000200090C2
:1036300002905038C0B2009D294600F0C3FA022023
:10364000294600F0BFFA10242046294600F0BAFAB5
:10365000E14E403E04960127304621463A46FFF7A8
:1036600042F9DD4839463A46FFF73DF930462146F2
:103670002A46FFF738F9D84839462A46FFF733F982
:1036800078242E46E0B2C20910210498FFF72BF9E6
:103690000127D14D284639463A46FFF724F9002242
:1036A000284639461546FFF71EF9701C6400072EA0
:1036B0000646E7D31021012704983A46FFF713F98D
:1036C000C54C204639463A46FFF70DF920463946A3
:1036D0002A46FFF708F94024E0B2C20910210498F5
:1036E000FFF701F90127BC4839463A46FFF7FBF8D6
:1036F0000026B94839463246FFF7F5F8681C6400E1
:10370000072D0546E8D31021012404982246FFF72F
:10371000EAF8B14D284621462246FFF7E4F828464C
:1037200021463246FFF7DFF83046354601960390D2
:10373000C000EF4908180299475CA74EF8B2C209C9
:1037400010210498FFF7CFF8012430462146224685
:10375000FFF7C9F8002230462146FFF7C4F8681C7D
:103760007F00072D0546E9D3102101240498224645
:10377000FFF7B9F8304621462246FFF7B4F8002299
:1037800030462146FFF7AFF80398401C8028019D82
:10379000CDD110240022049E30462146FFF7A3F825
:1037A00001278D4839463A46FFF79DF830462146B5
:1037B0003A46FFF798F80298401C082800D037E7EF
:1037C0000920C2018248CA49FCF7DAFC05B0F0BD05
:1037D000E8040020F0B585B000237D4CC44DD9002D
:1037E0006218125C6918095C914205D15B1C59B2E0
:1037F0000029F4D505B0F0BD02905038C0B20027C2
:10380000394600F0DFF90220394600F0DBF91026D6
:103810003046394600F0D6F96F4D403D0124284628
:1038200031462246FFF75FF86B4821462246FFF7F4
:103830005AF80495284631463A46FFF754F8664848
:1038400021463A46FFF74FF87825634E0397E8B2D2
:10385000C20910210498FFF746F80127304639467F
:103860003A46FFF740F80024304639462246FFF733
:103870003AF803994F1C6D000729E7D3102101275F
:1038800004983A46FFF72FF8534D284639463A46F2
:10389000FFF729F8284639462246FFF724F8402545
:1038A0004D4EE8B2C20910210498FFF71CF8012719
:1038B000304639463A46FFF716F800223046394678
:1038C0001746FFF710F8601C6D00072C0446E8D37C
:1038D00010210124049E30462246FFF704F83E4D95
:1038E000284621462246FEF7FEFF284621463A4654
:1038F000FEF7F9FF16E01021012430462246354636
:10390000FEF7F1FF344E304621462246FEF7EBFF2C
:10391000002230462146FEF7E6FF049F7F1C802FE1
:103920002E4642D00497F90029484018029A855C37
:103930006F4B59188F5CAF4217D10027E9B2CA0903
:1039400010213046FEF7CFFF0124234821462246AE
:10395000FEF7C9FF002220482146FEF7C4FF791C6C
:103960006D00072F0F46E9D3C5E78018039088182C
:1039700001900025F9B2CA0910213046FEF7B3FFC5
:103980000124F64821462246FEF7ADFF0022F34807
:103990002146FEF7A8FF691C7F00072D0D46E9D3DD
:1039A00001990978039A1170A5E710240022304686
:1039B0002146FEF798FF0127E84839463A46FEF7C8
:1039C00092FF304621463A46FEF78DFF05B0F0BD26
:1039D00068090020E804002080080140F0B58AB0A2
:1039E00006910590082B03D10624002C0AD175E01E
:1039F0005907D808002900D0401C59084143CCB2CF
:103A0000002C6BD00F98099058080290203AD0B241
:103A1000002501900001334908180090059A04938D
:103A2000039404E00246089D6D1CA54256D0082B65
:103A3000089504D10620019948432C490EE0182B23
:103A400008D0102B48D00C2B48D10C2001994843AA
:103A5000254903E0242001994843214908184019C9
:103A60000792D6B20478002306990DE0099A002A3D
:103A700016D0F2001E4DAA18D55D9D43D555431CA6
:103A8000491C6408072811D2184607270F40012354
:103A9000BB40CFB2FF08E207E8D0099A002AE8D07D
:103AA000F200134DAA18D55D1D43E7E70798401CA7
:103AB000049B082B039CB5D0C1B2059A891A029ABF
:103AC0009142089D02D1069A08320692029A9142CA
:103AD000059AA9D00246A7E70098C0E70AB0F0BD52
:103AE000A2830008B27D00083E790008167700081E
:103AF000E8040020F0B585B002AC07C4002B36D036
:103B00001C460A9D6808082D00D1801C01900B9F5F
:103B1000002610E0009730200143CAB2019870439C
:103B200002994018C0B203992B46FFF757FF761C45
:103B3000F0B2A0421BD2F0430019010606D00121C9
:103B40000A225143401E0206FAD100E001210498E6
:103B5000FCF7A0FD0A21FCF79DFD0029DAD10097B2
:103B60000198704302994018C0B23022DBE705B0DB
:103B7000F0BDF0B583B00646177838462038C0B29D
:103B80005E281CD8082B01D05D0800E006250898A7
:103B90000190541C029501980090F0B2FAB20D46C3
:103BA0001F46FFF71BFF3B462946029D7619601C06
:103BB00027783A46203AD2B25F2A0446EBD303B0C4
:103BC000F0BD0000F0B583B000910190634F3D4619
:103BD000403D10240126284621463246FEF783FE4A
:103BE000384631463246FEF77EFE002702952846CB
:103BF00021463A46FEF777FE584831463A46FEF7E8
:103C000072FE7824554EE0B2C20910210298FEF7E8
:103C10006AFE0125304629462A46FEF764FE002248
:103C200030462946FEF75FFE781C6400072F0746E2
:103C3000E9D31021012502982A46FEF754FE474C8D
:103C4000204629462A46FEF74EFE002720462946F2
:103C50003A46FEF748FE0098002818D040243F4E10
:103C6000E0B2C20910210298FEF73DFE0125304660
:103C700029462A46FEF737FE002230462946FEF73F
:103C800032FE781C6400072F0746E9D316E00024B3
:103C9000324E1021002502982A46FEF724FE012705
:103CA000304639463A46FEF71EFE304639462A4629
:103CB000FEF719FE601C072C0446EAD310210125EB
:103CC00002982A46FEF70FFE244C204629462A4633
:103CD000FEF709FE0027204629463A46FEF703FE76
:103CE000019C1E4EE0B2C20910210298FEF7FBFDB6
:103CF0000125304629462A46FEF7F5FD00223046CA
:103D00002946FEF7F0FD781C6400072F0746E9D32B
:103D1000102101910127029C20463A46FEF7E3FD5F
:103D20000E4E304639463A46FEF7DDFD0025304658
:103D300039462A46FEF7D7FD2046019C21462A46F1
:103D4000FEF7D1FD304639463A46FEF7CCFD0298E3
:103D500021463A46FEF7C7FD03B0F0BD800801409A
:103D6000401E41424141080201210902024A1368F2
:103D70008B43181810607047007000400A48417863
:103D800040220A43427070470120C006054908607E
:103D9000BFF34F8FBFF36F8F0348417880220A43F0
:103DA0004270704780E100E020020020054A0029AF
:103DB00003D011680143116070471168814311609D
:103DC0007047C04614100240054A002903D011680C
:103DD0000143116070471168814311607047C0460C
:103DE0001C100240054A002903D0116801431160EC
:103DF00070471168814311607047C0461810024037
:103E0000054A002903D01168014311607047116809
:103E1000814311607047C0460C10024080B50648CF
:103E20000068002800D080470220FEF7F1FE042041
:103E3000FEF7EEFE80BDC046E812002080B50648C1
:103E40000068002800D080470120FEF7E1FE042032
:103E5000FEF7DEFE80BDC046EC120020B0B50C4679
:103E6000054600F069FDA020204300F0ADFD280AC2
:103E700000F0AAFDE8B200F0A7FD00F05DFDA12072
:103E8000204300F0A1FD00F025FD044600F07CFD7C
:103E90002046B0BD10B5D84C23880E4A1A40228067
:103EA0008A4212D2A18865290FD264215143081891
:103EB000208002F0F9FEA28820882169C91C022313
:103EC00000F0F4F902F0F1FE01E00220207600207B
:103ED000A08010BDFF0F00001D480188A0220A43EA
:103EE0000280C84801882D200001124A91420246F2
:103EF00000D00022104B994200D01046EA490880B9
:103F00007047C0461248018805220A430280BD4816
:103F100001880748074A914201D0002200E0421D73
:103F2000054B994200D01046DF4908807047C046D3
:103F30000380FFFF464D000054430000DA4864212F
:103F40000180A520000202490A8802430A807047C6
:103F50009811002070B500290BD0CB4A0B4604788D
:103F6000D5886E1CD680166974555B1E401C002BCC
:103F7000F5D1F4480181FFF76FF970BDF0B581B05C
:103F80000D460B4C0026266005220223214600F038
:103F90008DF9277904212046FCF7B4FD874201D131
:103FA000012600E0256003480660206801B0F0BDEE
:103FB00060150020A8120020F0B581B0E14CA08867
:103FC000022800D274E03C4EEF4F8D4D02E0A088F5
:103FD00001286DD90220208121888A19092A17D841
:103FE0007A4412795200974407090B0D0F110413FC
:103FF000133B00F0CDF9EAE7288840E068883EE00E
:10400000A8883CE0E8883AE0288938E0688936E00A
:1040100000223A80274A914232D30A0A802A47D89E
:10402000244A6C3292B291422AD8224A5218143A47
:1040300091B2264B5943490CC04348438018714AFA
:1040400012881E4B9A421ED01D4B9A4218D149002D
:10405000214A525A3A6080B202281BD11F4825E0FB
:10406000684800881549884205D01549884205D11D
:104070001548008803E01348008800E000203880DD
:10408000FDF74EF8A3E74900114A525A3A6080B250
:1040900002280AD0012806D00028F1D1042020816E
:1040A000FDF73EF893E77888E9E70A48405AE6E7E3
:1040B00001B0F0BD0A8000000080FFFF324E00001A
:1040C000314E0000961100209A110020ABAA00008A
:1040D0002000002068000020F80E0020400F002083
:1040E000F0B581B0F44CA088022844D3FB20C50170
:1040F000224EA54F04E000F045F8A08801283AD9E7
:104100002088B042F7D33146703189B2884221D23B
:1041100008E048005E49085A3880FDF701F8A08899
:104120000128EAD90220208120882918703189B21B
:104130006F29EED931466F3189B2884218D80020F4
:10414000EAE788000E4908583860FCF7E9FFA088C4
:104150000128D2D9042020812088411989B20F2951
:10416000EFD93146EF3189B2884201D80020EBE720
:104170000020A080C1E701B0F0BDC0461082000061
:10418000A0010020F0B581B0CB4CA088022831D32B
:104190001A4D7D4EF74F05E03080FCF7C1FFA08837
:1041A000012827D902202081208841190B2913D802
:1041B0007944097949008F44090C0F0F0F0F0F0F35
:1041C00014171A05CF204000385AE5E70D4800883B
:1041D000E2E700F0B9F8DFE7000A82280AD80020F9
:1041E000DAE7FFF78FFED8E7FFF776FED5E7FFF7B0
:1041F000A5FED2E701B0F0BD24020020FE7DFFFF46
:1042000040020020880F0020F0B581B0AA4EB0888F
:10421000022836D31D4F5C4C1D4D05E02080FCF775
:104220007FFFB08801282CD9022030813088C11945
:10423000122913D87944097949008F440C0F0F14BF
:10424000171A0F0F0F0F0F1D0F0F0F0F0F0F090072
:104250008820285AE2E713480088DFE7000A84280C
:104260000FD80020DAE70E480088D7E70B4800880F
:10427000D4E70C21084801E00A210648FFF76AFE4E
:10428000CFE701B0F0BDC04624020020007CFFFF54
:10429000FA0D002054740008287400085A150020F4
:1042A000541500209211002068150020F0B581B04F
:1042B0001E4614460D46074600F03EFBA020304344
:1042C00000F082FB380A00F07FFBF8B200F07CFBC4
:1042D00000F032FBA120304300F076FB00F0FAFA48
:1042E0002870022C0AD36D1C012600F0BBFA00F0E6
:1042F000F1FA28706D1C761CA642F6D300F044FB40
:1043000001B0F0BDB0B502F0CFFC6B4CA2882088A4
:104310002169C91C0423FFF7C9FFA088411EA180A1
:1043200020698AB21218D578C01CC9B2FCF7EAFB22
:10433000854204D12069A1880818AA21C17002F021
:10434000B4FCB0BD2402002001207047F0B581B05C
:1043500000910D4C00272780032202262146334678
:10436000FFF7A4FFA57820463146FCF7CBFB85423A
:1043700003D10020A070012701E0009820800348AD
:104380000760208801B0F0BD68150020A812002049
:1043900010B54948C288511CC180036912490C7884
:1043A0009C54C288531CC38003694C789C54C288B7
:1043B000531CC38003698C789C54C288531CC380EF
:1043C0000369CC789C54C288531CC38003690C7960
:1043D0009C54C288531CC3800369497999540621AF
:1043E0000181FEF739FF10BD8E15002010B504467F
:1043F00000F0A2FA3E2000F0E7FA204600F0E4FACE
:1044000000F09AFA3F2000F0DFFA00F063FA044669
:1044100000F028FA240200F05DFA241800F042FAB5
:1044200000F0B2FA204610BDF0B581B0214C2078E2
:10443000FE21009108402070812040002518FDF7E2
:10444000E5FB1D4FA61C3E617D611C48205CB881C8
:10445000FEF7C2FE002814D0FEF70CFE1848FEF747
:104460008BF9B87A174960542078022101432170F2
:10447000FCF7FAFF0020144A0146FDF727F801B0C7
:10448000F0BD207800990840207000201521FCF72D
:1044900045FF0B4C2661207840010C49421821460B
:1044A0000C312046FDF7F4FF2046FEF75BF901B022
:1044B000F0BDC0468E0F0020240200200202000042
:1044C000080100200302000035120008009002409D
:1044D000F0B581B00A4D00242C606C603D4E27463B
:1044E000204621460A222346FBF732FEF25D801861
:1044F00061417F1C0E2FF5D103C501B0F0BDC04650
:1045000090120020F0B581B09048002282831A49B1
:104510000A60D34B1C88022C04D31346022C04D20D
:104520000B2503E00323022CFAD30825294EF75C60
:104530000A246243D2195B1C9FB2BD42F7D10A60C4
:104540007219858B0023D65C6543AD195B1C032B68
:10455000F9D1858308687D21CA00002421462346BD
:10456000FBF7F6FDAAB2054B80181860614159604F
:1045700001B0F0BD4002002080120020781200201F
:1045800010B513490B780F201C090340114A5370D2
:1045900014704B781C090340D37094708B781C09FD
:1045A000034053711471CB781C090340D37194718B
:1045B0000B791C090340537214724B791C09034098
:1045C000D3729472C979084050730809107310BDF2
:1045D000EC0D0020F401002010B507490A68012302
:1045E0009A430A600A68802414430C608860086853
:1045F0001843086010BDC046000C0040F0B581B003
:1046000000905F20C7430F4300F0BEF9072401204C
:1046100002F038FB00F090F9FDB2284600F0D4F922
:10462000064600F0B1F9002E03D0601E002C0446AF
:10463000EDD100F081F9284600F0C6F9009C200A6F
:1046400000F0C2F9E0B200F0BFF901B0F0BD000027
:10465000F0B585B0312000010221FFF777FE012778
:104660007C026B480078394908531121C943153839
:10467000884267D303204002674D0722022302903D
:1046800029460192FFF712FEAE7906212846FCF773
:1046900039FA86420FD169885D4B1980A988598003
:1046A0000021A97129882A4A11801968294A1160B4
:1046B000864247D106E0264900220A8025490A6041
:1046C00086423FD1E748005B022839D3214C03974B
:1046D000FEB2019A104670430299401802232946FF
:1046E000FFF7E4FDAF7906212846FCF70BFA7100CD
:1046F000174A5118049787420DD16A88444B1A8093
:10470000AA885A80B2001B68124EB3500022AA71C8
:104710002A880A8004E0B20000230E4EB3500B80BA
:1047200004998142039F0DD103CC083C814209D9F1
:1047300001204002CB49085A241D7F1C8742C6D362
:1047400005B0F0BDFCF7DEFE05B0F0BD4002002074
:10475000EC1100209C110020F0B581B00720000270
:104760002B4D0222009029461346FFF79FFD6E78DD
:1047700001212846FCF7C6F9864207D12878254C46
:1047800020802121C9432538884213D22448254955
:1047900001812549C1802549818025494180002129
:1047A00001801C48052202801C4801604160018193
:1047B00001B0F0BD20880028FAD00020E24D074665
:1047C0000BE04A000020154B98524900144A505201
:1047D0007F1CF8B221888142EAD905225043009912
:1047E0000818801C80B202232946FFF75FFD2E794E
:1047F00004212846FCF786F9F9B28642E1D1480047
:104800002A88064B1A52002028716888DDE7C046C6
:10481000681500209A11002060150020400F00202C
:10482000F80E0020204E0000983A000010270000EB
:104830008813000009490988022908D001290BD1F1
:1048400007490988002907D1C01C80B27047044974
:104850000988012900D1C01C80B27047B200002035
:10486000B0000020F0B581B0784C1025002620461D
:1048700029463246FEF737F800BF4034012720466C
:1048800039463A46FEF72FF800BF204639463246F1
:10489000FEF729F800BF6D4829463A46FEF723F88F
:1048A00001B0F0BDB0B50A4C2046403810210125BA
:1048B0002A46FEF718F800BF204629462A46FEF78A
:1048C00012F800BF002220462946FEF70CF8B0BDC2
:1048D00080080140F0B581B05C4C04252046294693
:1048E000FCF72CFF20462946FCF749FF0025082449
:1048F0000095564F3D464035012628463146324602
:10490000FDF7F1FF00BF10213846FDF7E5FF074630
:10491000002228463146FDF7E6FF781E87410098C1
:104920004000C51900BF641EE2D104214748FCF7CE
:104930000EFFE8B201B0F0BDF0B581B0434E344691
:104940004034002520462946FCF701FF042130466B
:10495000FCF7FDFE102601273C4831463A46FDF79C
:10496000C2FF204639463A46FDF7BDFF374831467B
:104970002A46FDF7B8FF00BF204639462A46FDF714
:10498000B2FF01B0F0BDC046F0B581B02F4E403649
:1049900001250027304629463A46FDF7A4FF00BF0F
:1049A00010242A4821463A46FDF79DFF00BF3046B5
:1049B00029462A46FDF797FF244821462A46FDF757
:1049C00092FF01B0F0BDC046F0B581B006460824A4
:1049D000F0B2C20910211D4D2846FDF784FF403575
:1049E0000127284639463A46FDF77DFF00BF0022E1
:1049F00028463946FDF777FF00BF641E7600002C7D
:104A0000E6D104260096114C20463146FCF796FE6E
:104A100020463146FCF7B3FE0127284639463A4680
:104A2000FDF761FF00BF10212046FDF755FF064648
:104A3000002228463946FDF756FF20460099FCF72C
:104A400086FE701E8641304601B0F0BD4008014030
:104A500080B5FF205E303C21FFF778FCDE21AC4AB8
:104A6000505280BD40020020B0B5934DA87A00019D
:104A7000924C607169782A78120189182170E9785E
:104A8000AA7812018918617069792A791201891846
:104A9000A170E979AA7912018918E170697A2A7AF4
:104AA000120189182171E97A0818607106212046DF
:104AB000FCF728F8A071687B297B09014018E07198
:104AC000B0BDC04670B5A04905220A763F4A1268BB
:104AD0003F4B9A4205D03F4B9A4202D03E4B9A42FE
:104AE00004D13E4A002313800B7603E000228A8023
:104AF0007B4B1A8004220A818A88032A06D87848C8
:104B0000002202808A800320087670BD00220A7687
:104B1000734A01231380CA88551CCD800B699E5CA3
:104B2000094CE670961CCE80ADB25D5DA570D51CBB
:104B3000CD80B6B29E5D6670121DCA80A9B2595C66
:104B400021702168016070BD601500200148024994
:104B500001807047A4120020FFFF000070B57A4961
:104B600005220A76194A1268194B9A4205D0194B48
:104B70009A4202D0184B9A4204D1184A002313805B
:104B80000B7603E000228A80554B1A8002220A81AC
:104B90008A88012A06D85248002202808A8003208F
:104BA000087670BD00220A764D4A01231380CA8818
:104BB000531CCB800C69A55C094E7570921CCA8091
:104BC00099B2615C31703188018070BD4C15002054
:104BD00055AA00003331303244524953220200209A
:104BE00068150020F0B581B03148002404803148B8
:104BF0000460314E70783178090140182F4D2870CB
:104C0000F078B1780901401868707079317909013C
:104C10004018A870F079B17909014018E870707AED
:104C2000317A090140182871B07A0001F17A081828
:104C3000687106212846FBF765FFA87120490C60C2
:104C400033488483727B337B1B01D218EA711D4A7F
:104C50001388022B04D32246022B04D20B2503E037
:104C60000322022BFAD30825B75C0A235C43E4191C
:104C7000521C97B2BD42F7D10C6071190022164642
:104C80008D5C5E437619521C032AF9D186837D2000
:104C9000C2000025204629462B46FBF759FAB2B23E
:104CA000094B801818606941596001B0F0BDC046D9
:104CB00074120020B0120020F4010020EC0D00203E
:104CC00080120020B000002078120020062803D3B4
:104CD000034800220280084640000249085A7047F3
:104CE000DC1200206A74000810B5194C2078FC21F1
:104CF00001402170A4200649085A8000054908583F
:104D0000FCF73EFB2078FE210140217010BDC0461B
:104D1000400200200091000880B50A48FDF72CFDF4
:104D20000948807A09490A4A5054107802210143FF
:104D30001170FCF799FB0020064A0146FCF7C6FB00
:104D400080BDC046080100202402002003020000AC
:104D50008E0F002035120008F0B581B004460F4DCB
:104D60002846FDF72BFE6E46002737703846FDF7C4
:104D7000F1FE77800220707028463146FDF740FE34
:104D8000012628463146FDF72DFE70075F49086071
:104D900028462146FDF768FE01B0F0BD000C00403A
:104DA000F0B581B004460F4D2846FDF707FE6E466C
:104DB000002737703846FDF7CDFE778002207070EF
:104DC00028463146FDF71CFE012628463146FDF7F0
:104DD00009FEB0064D49086028462146FDF744FE0D
:104DE00001B0F0BD200C004070B594202B49085A4A
:104DF000411E00243F2900D926E020467944097944
:104E000049008F44301F25272525252925252525BF
:104E10002525252B2525252525252525252525253C
:104E20002525252D2525252525252525252525252A
:104E30002525252525252525252525252525252522
:104E40002525252F01200EE0802801D107200AE02A
:104E5000052008E0022006E0032004E0042002E030
:104E6000052000E006200E4E7081022520462946CE
:104E7000FBF752FD0B480178FE220A4002707D20AC
:104E8000400200F013F83348074A294600F084FB3B
:104E9000B4807480FCF7F4FC70BDC046FA0D0020AD
:104EA000F012002020020020893D0008F0B583B0F8
:104EB00006460027029714480190264C01A9204677
:104EC000FDF7EAFE7D204002864200D3064601251A
:104ED000002E284600D030466063676202212046DB
:104EE0002A46FDF7CDFEE80608490860FF200006C7
:104EF00007490A688243A807101808602046FDF792
:104F0000F7FE03B0F0BDC046FB0000FA00E100E090
:104F100018E400E0024801680122914301607047F3
:104F200008A50240B0B50B4C2046FDF7E7FE012076
:104F3000C00609490860BFF34F8FBFF36F8F472545
:104F400020462946FDF798FE002220462946FDF717
:104F500097FEB0BD002C014080E100E080B5FDF778
:104F60000FFD80BD10B581000A4A52580A4B1A60E5
:104F70000A494A8042000A4CA25A0A805A888A800A
:104F80000722504303235B02C018022301F07EFD79
:104F900010BDC0469C11002068150020601500203F
:104FA000EC11002080B5FDF7F7FC80BD80B584B022
:104FB0000020039002900920019004200090684690
:104FC0000349FDF757FD002800D0FEE704B080BD7F
:104FD000FFFF000080B582B01C4908680007800F01
:104FE00000905A48009A032A0BD8C0467A44127996
:104FF000520097440104080B0A68520401D4144A71
:1050000006E0019005E07D22120201E00122D203B8
:10501000019209680906090F00910099082901D237
:10502000002106E0009A00990B2A01D8C91F00E070
:10503000891F00910199009AD140434A116011687B
:10504000FDF75AFC4249087002B080BD04100240CE
:105050000048E801B0B582B06C460020A071FF2086
:105060000230A0800B4800900B4D28462146FDF7EA
:10507000AFFB284640302146FDF7AAFB20881E21C1
:1050800088432080803528462146FDF7A1FB02B0E9
:10509000B0BDC046FFFF010000080140F0B581B07F
:1050A000664800240460214F3C808480022520460D
:1050B0002946FEF7D3FE401CC6B2204631462A469A
:1050C00001F0ECFA20462946FEF7C8FE864205D0DC
:1050D00001205A49487079780143797000240425E9
:1050E00020462946FEF7BAFE401CC6B2204631468D
:1050F0002A4601F0D3FA20462946FEF7AFFE864243
:1051000005D001204D4988707978014379700620D7
:10511000FFF76CF9542806D0012048494871787887
:1051200040210143797001B0F0BDC0465615002002
:1051300005480649016006480221017005480168DA
:1051400001220A4302607047100000200024F4008E
:10515000000000201410024070B53548002404807F
:10516000FBF740FD33480460334804803348046053
:105170004460846032484021FBF729F8A425994E09
:1051800003207053A22101227252A02174522921BE
:1051900049029E22B152572189007452DA21745279
:1051A000D8217452C0217452BE217452BC21745251
:1051B000B821745223490C6023490C6023490C60C8
:1051C00023490C6080490A78DF2313400B70B349F0
:1051D0000A78FA2313401A1D0A70C8217452CF218D
:1051E00049007452C12149007452C0013452194817
:1051F0000460194804801948046044601848048019
:105200001848017810220A430270FCF7F5F9FFF7FD
:1052100045FF00F02FF8705B80001349085800F03C
:105220000DFAFFF761FD11481149018070BDC046BC
:10523000AC1200208812002016120020E401002089
:10524000A8150020D4120020CC120020E40E00206B
:10525000EC0E0020E80E00207412002078120020CE
:10526000A015002014120020009100085C150020F9
:1052700055AA0000F0B581B0534C2078BF21014001
:105280002170FCF7D7FDFCF7F3FC504A1088504919
:105290000880504D2988118040004F4A105AC0099B
:1052A0004E4B18804800105AFFF796F92078DF21FE
:1052B000014021704A4F0126000701D5304600E029
:1052C000388A2880FBF78EFC1020464C0C220223E3
:1052D0002146FEF7EBFFFF25043528463146FFF750
:1052E00035F8A221605228461E303F49FFF72EF8BC
:1052F000B6216052FBF778FCFBF774FCF1032846FB
:105300002730FFF723F8BC216052388A2F490880E4
:105310003146FFF7DBFCCA216052284624300426C0
:105320003146FFF713F8314908803146FFF7CEFCCC
:10533000BA21605228460C302D49FEF71FFEAC21E1
:1053400060522C4F38607988AA22A1522A490860FD
:10535000A81D00263146FEF711FEA82160523860D4
:105360007988A622A15225490860FBF73BFC284614
:1053700057300321FEF7EAFFDC21605228466F30E8
:105380003021FEF7E3FFEC216052284672301A21EB
:10539000FEF7DCFFEE216052753528463146FEF7F8
:1053A000D5FFF021605200F081F9FCF7E1FBFFF737
:1053B0004FFBFFF74DF9FFF7CFF9FFF7C7FBFCF7FE
:1053C00033FC01B0F0BDC04692110020441500200E
:1053D00046150020481500205E7400088C1500203A
:1053E000FA0D00204002002006040000E412002014
:1053F000C027090068150020D0120020D812002014
:1054000010B5264C607840060BD5FDF703FDFDF77F
:105410004DFFFBF7E7FBFFF7E7FC6078BF2101409A
:1054200061701F480078C00701D0FEF7FDFF1D48DE
:105430000078401E414241411B480078401E4242D4
:1054400042410A43012A1ED1C449087800280BD0E2
:105450000020087016490A78521CD3B2032B00D8DA
:105460001046087000F07CF912480178002914D029
:105470000021017000F074F90F4C207800280CD145
:10548000FBF75AFA07E0094C2078002805D1FDF710
:1054900085FFFEF7C9F80120207010BD2002002012
:1054A0008E0F0020A21500209A120020E80D002087
:1054B000941100201812002099120020B0B5114C50
:1054C0002568E80704D052480068002800D08047CB
:1054D000A80704D551480068002800D08047680715
:1054E00004D54D480068002800D08047680604D5E0
:1054F00048480068002800D080471648A84320602C
:10550000B0BDC046102C0140B0B5114C2568E8076D
:1055100004D03B480068002800D08047A80704D585
:105520003A480068002800D08047680704D536480C
:105530000068002800D08047680604D5314800681C
:10554000002800D080470348A8432060B0BDC04673
:1055500010000040FFFF000010B50648006800285A
:1055600000D0804701242046FCF758FF2046FCF776
:10557000EBFE10BDF00E002010B5064800680028B4
:1055800000D0804702242046FCF748FF2046FCF765
:10559000DBFE10BDF40E002010B501239C07A042D5
:1055A0000BD0164CA04227D1D80603290EDC0129C6
:1055B00018D0022920D119491BE0180703290BDC58
:1055C000012911D0022917D1104912E004290DD068
:1055D000402911D10F490CE0042909D040290BD1F1
:1055E000084906E00A4904E0054902E00A4900E0EA
:1055F00005490B4B18600A6010BDC046002C0140E5
:105600008815002084150020801500207C150020BE
:105610007815002074150020701500206C150020EE
:1056200000E100E010B5194C04212046FDF76EFBA7
:1056300002212046FDF76AFB10BDC046F0B587B0D9
:10564000019005AD0327AF7101200002A8800D482D
:1056500005903F4E30462946FDF7BAF8AF71002459
:10566000AC800948059030462946FDF7B1F802A9FB
:105670000C810397019802900448FDF75DFB07B089
:10568000F0BDC046020000010400010100380140E5
:1056900010B5054C04212046FDF738FB02212046B9
:1056A000FDF734FB10BDC0460048004010B5132084
:1056B000000101242146FEF749FEC0210C4A505248
:1056C000401E83B2032B06D200B241000948405A63
:1056D000094A545A01E05452022008490C800849F2
:1056E0000C8008490880084908800849088010BDD6
:1056F00040020020307200082A7200088412002044
:1057000086120020B4000020B2000020B00000206B
:1057100010B50F4801242146FDF7DEF80D490A783F
:10572000002A04D0012811D1002008700BE00028C5
:1057300009D109480288521C028090B2032805D37F
:10574000064804700C7004480021018010BDC0465A
:1057500000080140F80D0020F60D0020AE120020D8
:10576000F0B58BB0AD480068FAF780FF0025AC4B70
:105770002A46FAF797FE07460E46AA480478012CF7
:1057800007D0022C08D0032C0ED101208207A74B92
:1057900004E00022A64B01E00022A34B384631462C
:1057A000FAF718FE07460E46032C24D87C442479C9
:1057B0006400A7440128496B05204207A54B3846E1
:1057C0003146FAF755FDFAF713FF0A900024A24B71
:1057D000384631462246FAF7FDFD994B2246FAF744
:1057E00047FDFAF705FF0A21FAF754FF05916620F5
:1057F00008909BA025E07E2008908E480490059597
:1058000009950A9563E005204207924B38463146D8
:10581000FAF72EFDFAF7ECFE0A9000248E4B38467C
:1058200031462246FAF7D6FD854B2246FAF720FD8F
:10583000FAF7DEFE0A21FAF72DFF05915A200890AB
:1058400086A00490012041E0072042077A4B3846A9
:105850003146FAF70DFDFAF7CBFE0A900024704BA3
:10586000384631462246FAF7B5FD754B2246FAF71F
:10587000FFFCFAF7BDFE7D21C900FAF70BFF059189
:105880004E20089071A0049003201FE007204207DB
:10589000694B38463146FAF7EBFCFAF7A9FE0A9055
:1058A0000024664B384631462246FAF793FD644B96
:1058B0002246FAF7DDFCFAF79BFE6421FAF7EAFECE
:1058C00005914E2008905FA00490022009900126C7
:1058D0000A980028354609D000260A9C0A2120464D
:1058E000FAF7D8FE761C092C0446F7D800201427B6
:1058F0007E222C23039039460797FDF75FFD009524
:105900000695182408983946049A2346FEF731F97B
:10591000009401950B20C04301467143099A5043FE
:10592000089A871808970C3FC819C0B2F3B2079DB0
:1059300029460A9AFEF7DEF8069E0096F8B22E2255
:1059400029462346FEF74AF8009401960898C0B20B
:105950002946059A099BFEF7CDF84248C08B42497B
:10596000884201D904240FE04049884201D9032428
:105970000AE03F49884201D9022405E03D498842B6
:1059800001D8039C00E00124682000217E220C2322
:10599000FDF768FD692001217D220B23FDF738FD0D
:1059A000601E03281ED8C046784400794000874412
:1059B000130D0701792002217C220A23FDF752FDF5
:1059C0007420022177220A23FDF74CFD6F2002216B
:1059D00072220A23FDF746FD6A2002216D220A2366
:1059E000FDF740FD7E200324802209232146FDF798
:1059F00039FD0020FDF7EEFE0120FDF7EBFE022051
:105A0000FDF7E8FE2046FDF7E5FE0420FDF7E2FE87
:105A10000520FDF7DFFE0BB0F0BDC046E012002010
:105A200000408F4094110020FDB87E3FE17A843F12
:105A3000A7001E40189100084D62403F00005940E9
:105A40000000E03F6D62617200000000746F7272CE
:105A5000000000009999A93F000024406D636D008B
:105A600070610000A8150020D8AE00007DAA0000DB
:105A700023A60000C9A10000F0B581B07A487B4D93
:105A80000560B04C2288FF203230824235D27849FE
:105A90001BE05A005219603A12880A80E288531CAF
:105AA000E38023694E789E54E288531CE380236987
:105AB0000E789E54022222812288521C2280A388C2
:105AC0009B1EA38093B2834217D2A388022B00D2DD
:105AD000C7E093B292B22F2ADBD85A0052190123A1
:105AE0005B02D35A23811A46303A92B20646303EC0
:105AF000B6B2B242CDD30022CFE7A088022800D2AE
:105B0000AFE05D4F5A4E05E0FDF7A6FBA0880128E7
:105B100000D8A6E0022020812188C8193C2800D99D
:105B20005DE0C0467844007940008744671E7733C3
:105B30001E77331E77331E77331E77331E77331E5F
:105B400077331E77331E77331E77331E77331E77F6
:105B5000331E77331E77331E77331E77331E77332A
:105B60001E77331E77331E773300042020810120F7
:105B700040022A5A3F484018801C80B2404948439E
:105B8000400C824201D80021316080003E49085813
:105B9000306010E0012040022A5A3648081880B2CE
:105BA00037494843400C824201D8002131804000EF
:105BB0003449085A30802089002800D1A4E7012107
:105BC000E288531CE3808BB280B2C01A305C236938
:105BD00098542089491C8AB29042F1D294E7274810
:105BE000081805281AD8C046784400794000874430
:105BF00002090B0E10134B20C000DBE7012040020E
:105C0000285AD7E71A20D5E77D200001D2E71220D5
:105C1000D0E77D20C000CDE70C20CBE71B48084033
:105C200020800F2212030A40228101210B039A4295
:105C300009D003231B039A4208D049038A4210D19A
:105C40001449122206E012491A2203E04B21C9002E
:105C5000AB310C22424350182080FEF753FB00204A
:105C6000A08001B0F0BDC046E0010020400200204D
:105C700068150020CDFE0000D0FEFFFF00F1FFFF01
:105C8000ABAA0000EC1100209C110020FF0F0000C7
:105C90000331000003710000F0B59FB0294E7088F9
:105CA00001210491090205916D31884202D9022037
:105CB00030762BE0244909680022244F06E006AD27
:105CC000AC525B1C3380921C662A11D0338883420D
:105CD0000ED22F2B1C46F2D85C00641801256D02F1
:105CE000645B34813D19303DADB2BD42E7D2DEE7A1
:105CF00017480078002802D0164817490160002094
:105D0000308002903081307E002801D01FB0F0BD7D
:105D10000520C001039002E0307E0028F6D1FDF797
:105D2000B1FA0028F2D13088400006A9095A0A4683
:105D3000373A53089A2B00D9B4E108A352009A5A73
:105D40005200974424020020E0010020FEFE0000E3
:105D5000A61200204C15002055AA0000AA01AF0190
:105D6000AF01AF01AF01B501AF01CA01AF01AF0192
:105D7000AF01AF01AF01AF01AF01AF01AF01AF01A3
:105D8000AF01AF01AF01AF01AF01AF01AF01AF0193
:105D9000AF01AF01AF01AF01AF01DB01AF01AF0157
:105DA000AF01AF01AF01AF01AF01AF01AF01AF0173
:105DB000AF01AF01AF01AF01AF01AF01AF01AF0163
:105DC000AF01AF01AF01AF01AF01AF01AF01AF0153
:105DD000AF01AF01AF01AF01AF01AF01AF01AF0143
:105DE000AF01AF01AF01AF01AF01AF01AF01AF0133
:105DF0003E02AF014E02AF015B02AF01AF01AF0146
:105E0000AF01AF016902AF0179028D02AF019602C5
:105E1000AA02B402AF01AF01BA02AF01AF01AF01F4
:105E2000AF01AF01AF01AF01AF01FD020303AF014D
:105E3000AF01AF01AF01AF01AF010A0314031E03AD
:105E4000AF01AF01AF01AF01AF01AF01AF01AF01D2
:105E5000AF01AF01AF01AF01AF01AF01AF01AF01C2
:105E6000AF01AF01AF01AF01AF01AF01AF01AF01B2
:105E7000AF01AF01AF01AF01AF01AF01AF01AF01A2
:105E8000AF01AF01AF01AF01AF01AF01AF01AF0192
:105E9000AF01AF01AF01AF01AF01AF01AF01AF0182
:105EA000AF01AF01AF01AF01AF01AF01AF01AF0172
:105EB000AF01AF01AF01AF01AF01AF01AF01AF0162
:105EC000AF01AF01AF01AF01AF01AF01AF012803D7
:105ED000AF0138035F03AF017703AF01AF01AF013B
:105EE000AF01AF01AF01AF01AF01AF017F034101CE
:105EF0004101410141014101410141014101410192
:105F00004101410141014101410141014101410181
:105F10004101410141014101410141014101410171
:105F20004101410141014101410141014101410161
:105F30004101410141014101410141014101410151
:105F400041014101410141014101410141019203EE
:105F50005D01AF0180015D01AF0180015D01AF0115
:105F600080015D01AF0180015D01AF0180015D0134
:105F7000AF0180015D01AF0180015D01AF018001D2
:105F80005D01AF0180015D01AF0180015D01AF01E5
:105F900080015D01AF0180015D01AF0180015D0104
:105FA000AF0180015D01AF0180015D01AF018001A2
:105FB0005D01AF0180015D01AF0180015D01AF01B5
:105FC00080015D01AF0180017818811C318188B2A8
:105FD0004000094A101A0D2252018018074A106029
:105FE00003224A430399511889B20023059A00F00D
:105FF000E7FD022030818FE640020020E001002012
:1060000004984002F64A105A79182F3989B2F54A95
:106010004A43540CA04200D878E6F34D2846FEF7D8
:1060200051FDF2480088002800D16FE6A0002968E1
:10603000EF4A1150EF480178F7220A400270E0B2AF
:10604000FEF790FF68E604984002E54A105A791876
:10605000313989B2E34A4A43540CA04200D855E68C
:10606000E54D2846FEF77AFDE0480088002800D17B
:106070004CE62888E14A1118703989B2914200D261
:1060800044E66100DE4A5052E0B2FEF76BFFD948A9
:106090000178F7220A4002703EE6FA480E30FEF719
:1060A0005DFD39E6022030810020F949088033E6A1
:1060B000B188042900D229E606A9401840883D2865
:1060C00000D023E6F04D2846FEF7FCFC2868F14995
:1060D000884200D90FE200200EE2CF204500E94CB3
:1060E0006019FEF73BFDE948018848424841615B81
:1060F000C9087C2900D9DDE10021DCE1B18808294B
:1061000000D203E606A941184988572900D0FDE5C9
:1061100006A941188988582900D0F7E506A9401832
:10612000C088592800D0F1E5D74D2846FEF7CAFCB3
:10613000D94C2046FEF7C6FC08203081D3480088A1
:10614000002800D1E8E5296825681720D34A521BAA
:10615000884100D2E0E57D20C20000242846234685
:106160000194F9F7C5FF0090CD4A1060CD4A23464F
:10617000F9F7EEFF4019C3498883CB4C082201256B
:10618000009821462B46FAF7A7FFBE48808B0834BB
:10619000032221462B46FAF79FFF019C2046FEF77B
:1061A00049FB0546BC480560C04844730473C4728B
:1061B00040190B22BC49F9F7E3FF0B35B6480560DF
:1061C000C6E1B048A2300599C91CF7220123FBF7AC
:1061D0008DFCAE480088002800D19DE5FAF762FCEE
:1061E0009AE506A940184088842800D08EE5F74833
:1061F0000068059909314208F54809E006A94018E8
:106200004088862800D081E505990F31EF48A84ADB
:10621000002300F041FB7FE5EF48B63005992131BE
:10622000F84AFA2300F0CCFCEC480088002800D1A2
:1062300072E5FAF7D9FC6FE5CF204500E64C60190E
:10624000FEF78CFCE5480088002800D164E5625B1D
:10625000E4490888904200D080E1002101208CE1CF
:10626000DD48BC3005992A31E34AE44B00F0A8FC34
:1062700052E5CF204500D84C6019FEF76FFCD74897
:106280000088002800D147E5605BC021615A884240
:1062900000D141E5FAF7DEFC3EE5CF48C230059972
:1062A0003331D34AD34B00F08BFCFFF735FDF84870
:1062B000C43005993631CD4A68E0CF204500F44C12
:1062C0006019FEF74BFCC5480088002801D1FFF794
:1062D00023FD625BC34B18889042049802990ED04C
:1062E0009B1C0020C14304290BD09C1C491C1B880B
:1062F00093422346F7D1052900D20120491C0028EA
:1063000003D10020B54908800121E1484153B34839
:106310000088002801D1FFF7FFFCDC4801800598C8
:106320003F3000F001FCB0490882062803D300206A
:10633000AA49088001204000AA49085ACA213CE124
:10634000D348DC3005995A3104221FE0D048DE30B2
:1063500005995D31039A503218E0CD48EC3005992B
:106360007231F022302300F02BFCFFF7D5FCC84837
:10637000EE30059975312822012300F021FCFFF74A
:10638000CBFCC348F03005997831954A002300F0E2
:1063900017FCFFF7C1FCCF204400BD4D2819FEF7C4
:1063A000DDFB285B8B49884201D0FFF7B5FCFAF78B
:1063B000E5FBFFF7B1FCCF204400B54D2819FEF7EF
:1063C000CDFBF6480088002801D1FFF7A5FC285B2B
:1063D000012801D0FFF7A0FCFAF7F8FBFFF79CFCBF
:1063E00040020020ABAA000098150020DC1200201B
:1063F0009C11002020020020681500200BE70000FF
:10640000EC110020CF204400A14D2819FEF7A6FB77
:10641000E2480088002801D1FFF77EFC285B0228B3
:1064200000D1CEE0012801D0FFF776FC00F094FA0D
:10643000FFF772FCCF20400095490818FEF78EFB4D
:10644000FFF76AFCCF204400914D2819FBF7E6FACC
:10645000295BD048814201D0FFF75EFCCE49029A09
:106460000A80CB490860FFF757FC0498400288492E
:106470000818039990311422032300F0A1FBFFF7C1
:106480004BFCC0464002002098150020DC12002082
:1064900068150020FFE0F5059C150020FFE7764811
:1064A0008012002018FC0000E4010020F40100200C
:1064B000FFFFFF7F0121084301D0FFF72DFCFEF70E
:1064C0005FF82146524C002060732073E072485BF5
:1064D0004E4D2946083103220123FAF7FDFD08201D
:1064E000FEF7A8F9297A215421186A7A4A70AA7A03
:1064F0008A70C01C2AE00120A84909884A424A4102
:10650000024301D0FFF708FCFEF73AF828683F4D38
:10651000082201232946FAF7DFFD3D4C0020A07038
:1065200060702070FEF786F9297821542118EA79E5
:10653000CA71AA798A716A794A712A790A71EA78E4
:10654000CA70AA788A706A784A7008302E49086042
:10655000FEF748FBFDF7D6FFFFF7DEFB8B1C0020A4
:10656000C14304290BD09C1C491C1B889342234621
:10657000F7D1052900D20120491C002803D10020B1
:1065800086490880042142484153844800880028F5
:1065900001D1FFF7C1FB3D4801800598273000F08D
:1065A000C3FA17490880062803D30020E949088068
:1065B000042040000B49085ABA21354A5052FFF7CF
:1065C000ABFBFAF79FFFFFF7A7FBC046D0120020F6
:1065D000D812002055AA000040020020DC12002042
:1065E000C8AF00006A740008FA0D0020FFFF000029
:1065F00088B6000068680000A08F0000607000008E
:10660000E41200207C1500009C150020E40100200D
:10661000F401002070B586B01A48017801AC2170F1
:10662000417861708178A170C178E1700079207142
:1066300015480178A1724178E17281782173D949B6
:106640000D88D54A92890A804B78124E36680E60C2
:10665000C07860732273E673E37288786073487859
:10666000A07311212046FAF74DFA607412225543A7
:106670000948281880B20423214600F007FA0020B8
:1066800006B070BD8E150020EC0D002068150020AE
:10669000400200208812002003710000F0B581B094
:1066A00015460E460746194820210022FCF71BF923
:1066B0005F20C4432C43FEF73FF9E5B22846FEF7BE
:1066C00083F9380AFEF780F9F8B2FEF77DF9304613
:1066D000FEF77AF9FEF758F90727012000F0D2FA01
:1066E000FEF72AF92846FEF76FF90646FEF74CF941
:1066F000002E03D0781E002F0746EED12021012264
:106700000248FCF7F0F801B0F0BDC0464008014077
:10671000B0B50446D64D05202876D6480068D64A3E
:10672000904205D0D54A904202D0D54A904204D139
:10673000D448002202802A7603E00020A880D24AB2
:1067400010802888164A02402A808A421BD2A888D4
:10675000652818D200F0A8FA288864214143081956
:106760002880E9882A69511880B2AA88022300F09B
:106770008DF900F09AFA0020A8800A48017840229A
:106780000A430270B0BD022028760020A880B0BD68
:106790004C15002055AA000022020020DC12002027
:1067A000FF0F000058150020B0B5B1480621018147
:1067B0008188052904D80321017600218180B0BD9C
:1067C000C1884B1CC3800269555C864C65718D1C69
:1067D000C5809BB2D35C2371CB1CC380ADB2555D29
:1067E000E5700D1DC5809BB2D35CA3704B1DC380AB
:1067F000ADB2555D6570891DC18099B2515C217043
:106800000021616000881949401880B2184941434D
:106810004D0C184800881849884214D017498842FE
:1068200022D10522104668431849401880B202233D
:10683000214600F02BF968006188154A1152218821
:10684000144A1152B0BD0522104668430C49401845
:1068500080B20223214600F019F968006188094AD4
:1068600011522188084A1152B0BDC046F67F00007F
:10687000ABAA0000880F0020324E0000314E00000D
:10688000020800002000002068000020020700002D
:10689000F80E0020400F0020F0B583B00446F14808
:1068A00005250576F04D2D68F04EB54205D0F04E29
:1068B000B54202D0EF4EB54204D1EF4D00262E80F6
:1068C000067603E000258580EC4E358004250581A1
:1068D0008588032D09D8E94D00262E808680032562
:1068E0000576904227D903B0F0BD00250576E34D2B
:1068F00001262E80C588029101921A4623466C1CFF
:10690000C4800669715D374FF970A91CC180A4B2BB
:10691000345DBC70EC1CC48089B2715C7970291D37
:10692000C180A0B21C461346019A0299305C3870AF
:1069300038689042D7D89842D5D322688242D2D0C4
:10694000CE4801220280084600F02EF8206003B0F5
:10695000F0BDC046DC120020F0B581B00D20400132
:106960000D4908180D4C206000250D4EC44F705D78
:10697000216808803880032068430521C901401838
:1069800080B200F0D1F82068801E20606D1C302D90
:10699000EDD101B0F0BDC04640020020E001002072
:1069A000F873000868150020F0B581B00546009026
:1069B0000C4C04212046FAF7A5F820710526022781
:1069C0002846214632463B4600F060F80025256007
:1069D0000098214632463B46FDF768FC2571206849
:1069E00001B0F0BD60150020F0B583B014460B4631
:1069F00002469C4D052028769B4800689B498842AA
:106A000005D09B49884202D09A49884204D19A48CD
:106A100000210180297603E00020A88097490880A2
:106A2000032028769548002606802C81A888A0425D
:106A300002D2AE8003B0F0BD2E76E888296909182D
:106A4000022718460292224601933B4600F01EF8A8
:106A500001208A4908802E76E8880019E88001988C
:106A6000029922463B46FDF721FC03B0F0BDC0462B
:106A7000240200204C15002055AA0000333130328A
:106A80004452495322020020DC120020F0B583B0AA
:106A9000029300920C4606462248202100273A46DF
:106AA000FBF721FF5F20C54302980543FDF744FF34
:106AB000E8B20190FDF788FF300AFDF785FFF0B2DC
:106AC000FDF782FF0098002810D0054603E0641C03
:106AD0007F1CAF420AD22078FDF776FF761CB00605
:106AE000F5D1B0B20299FDF789FDF0E7FDF74CFF53
:106AF0000726019D012000F0C5F8FDF71DFF28467F
:106B0000FDF762FF0446FDF73FFF002C03D0701E27
:106B1000002E0646EED1202101220248FBF7E3FEBB
:106B200003B0F0BD40080140F0B581B00546544CBB
:106B3000022620463146F9F7E5FFA07003272846D4
:106B400021463A463346FFF7A1FF284621463A46FA
:106B50003346FDF7ABFB0020A070208801B0F0BDEC
:106B6000B0B54048062101818188052904D8032158
:106B7000017600218180B0BDC1884C1CC4800269AF
:106B8000555C0E4B1D708D1CC580A4B2145D5C70ED
:106B9000CC1CC480ADB2555D9D700D1DC580A4B2E6
:106BA000145DDC704C1DC480ADB2555D1D71891D36
:106BB000C180A0B2105C5871B0BDC0468E150020D7
:106BC000F0B583B01F460291044626480525057698
:106BD000254D2D68254EB54205D0254EB54202D033
:106BE000244EB54204D1244D00262E80067603E0C3
:106BF00000258580214E3580022505818588012D5F
:106C000009D81E4E002535808580032606769542DC
:106C100019D903B0F0BD00250576184D01262E8048
:106C2000C5886E1CC6800197076921467C5D144BA0
:106C30005C70AC1CC4800C46B0B2385C019F18700C
:106C40001D889542E5D8BD42E3D32088A842E0D014
:106C50000A48012101800298FFF766FF208003B0F7
:106C6000F0BDC046240200204C15002055AA0000AB
:106C7000333130324452495322020020DC120020CA
:106C80006815002000280ED0AD21C90000BF491EA4
:106C90000A04FBD100BF00BF00BF00BF00BF00BFA0
:106CA000401E0104F0D170477047704710B502468E
:106CB00001230A48824206D01B4CA2420AD19C06FC
:106CC0002030074A01E05C07034A1160FBF770FEC1
:106CD0000448046010BDC046C4120020000C0040EF
:106CE000C812002000E100E0FEF738F9FEF75EF977
:106CF000FEF7B0F9FF204830FEF752F80A480B497A
:106D0000FFF7D4FFFBF770F9FAF742FD08480021BE
:106D10000180FEF721FAFCF7CFFB06482021FAF7A5
:106D200016FDFEF76DFBFCE7200C00405133000818
:106D30005C150020000801400FB410B504A9074BF2
:106D400002AA039800F032F8044602A9002000F0DD
:106D500067FA204610BC08BC04B01847217200082E
:106D60002021020C01D010211046020A01D0104649
:106D70000839020901D01046091F820801D01046C7
:106D8000891E420801D0881E7047081A704702E029
:106D900008C8121F08C1002AFAD1704770470020A6
:106DA00001E001C1121F002AFBD17047FFB591B06D
:106DB0000F460546002606E025280AD0149A1399A6
:106DC00090476D1C761C28780028F5D1304615B008
:106DD000F0BD002400940121F34A029400E0044332
:106DE0006D1C2B780846203B98401042F7D128783C
:106DF0002A280ED0022128780246303A092A15D8CE
:106E0000009A0A235A43303A80180C436D1C0090B4
:106E1000F1E701CF0090002805DA01204003044388
:106E2000009840420090022004436D1C28782E28D0
:106E300015D10420044368786D1C2A280AD101CF9B
:106E40006D1C02900BE002990A2251433039401820
:106E50006D1C02902878014630390929F3D9287829
:106E60006C2810D006DC4C281AD068280ED06A286E
:106E700017D104E0742813D07A2812D110E0012031
:106E8000400504430CE00121090501E00321090547
:106E90000C436978814203D10120000524186D1C40
:106EA0006D1C287803906E281ED00CDC632831D02E
:106EB00004DC00288AD0582811D1B2E064287BD0A5
:106EC00069280CD178E073282DD004DC6F2870D0AD
:106ED000702804D1A7E075286CD078286BD0149A5C
:106EE00013999047761C62E06002400F022807D099
:106EF00003280AD0042838680AD006603F1D56E0EF
:106F00003868F11706604160F8E738680680F5E7F1
:106F10000670F3E73878694608740020487404A8BE
:106F20000390012003E0386803900020C0433F1D18
:106F300061070FD5002101E00199491C029A0191D6
:106F4000914213DA8142F7DB019A0399895C0029A7
:106F5000F2D10BE0002101E00199491C019181422D
:106F6000FADB019A0399895C0029F5D1019900980F
:106F7000139A401A00902146149B00F03BF90199A6
:106F80008019461807E0039803990078491C03917B
:106F9000149A139990470198401E0190401CF2D119
:106FA0002146149B139A009800F014F986196D1C61
:106FB00009E741E033E034E00A2000210490059124
:106FC0006002410F022905D001CFC2179446032960
:106FD00005D007E0FF1DFF08FF0003CF06E000B269
:106FE000C2179446042902D140B2C1178C46002230
:106FF0006146944506DA0A460021404291418C469A
:107000002D2102E0210504D52B216A4611760121AC
:1070100003E0E10701D02021F7E7019154E00A20C5
:107020000BE0102009E0102004900021042004430C
:1070300008200591029003E00820002105910490AA
:107040006002410F022905D001CF00229446032996
:1070500006D006E0FF1DFF08FF0003CF8C4603E0CB
:1070600080B2042900D1C0B20021019121072BD5A3
:107070000399702906D0049A1021059B4A401A43AF
:1070800005D00EE040216A461176012108E06146F4
:10709000014306D030216A461176039951760221C8
:1070A0000191049A0821059B4A401A430CD161467C
:1070B000014301D1610707D530216A4611760121CC
:1070C00001910299491E02910399582904D037A1D0
:1070D00003910FA90F910DE039A1F9E76146059BD6
:1070E000049AF9F705F8039B8C469B5C0F9A521E95
:1070F0000F92137061460143F0D10F9807A9081A47
:1071000020300390600704D50120000484430298D6
:1071100001E0012002900399884201DD401A00E05D
:10712000002041180290019809180098401A009018
:10713000E00306D42146149B139A009800F05AF8F5
:1071400086190020049008E006A9085C149A139997
:1071500090470498401C761C049001998842F3DB08
:10716000E0030CD52146149B139A009800F042F8D6
:10717000861904E0149A302013999047761C0299DE
:10718000481E02900029F5DC08E00F980F9900785E
:10719000491C0F91149A13999047761C0399481E25
:1071A00003900029F1DCFBE609280100303132337D
:1071B0003435363738396162636465660000000033
:1071C000303132333435363738394142434445461D
:1071D00000000000F8B5044600251E461746880446
:1071E00004D405E039462020B0476D1C641EF9D553
:1071F0002846F8BDFFB50446002581B01E46C803E9
:1072000001D5302700E02027880404D505E0384662
:107210000399B0476D1C641EF9D5284605B0F0BD32
:107220000A68531C0B6010707047010002000500D3
:1072300002000200030000070E091C1B1215383F54
:10724000363124232A2D70777E796C6B6265484F26
:10725000464154535A5DE0E7EEE9FCFBF2F5D8DF16
:10726000D6D1C4C3CACD90979E998C8B8285A8AF86
:10727000A6A1B4B3BABDC7C0C9CEDBDCD5D2FFF876
:10728000F1F6E3E4EDEAB7B0B9BEABACA5A28F88E6
:10729000818693949D9A2720292E3B3C35321F18D6
:1072A000111603040D0A5750595E4B4C45426F6846
:1072B000616673747D7A898E878095929B9CB1B646
:1072C000BFB8ADAAA3A4F9FEF7F0E5E2EBECC1C6A6
:1072D000CFC8DDDAD3D4696E676075727B7C515696
:1072E0005F584D4A4344191E171005020B0C212606
:1072F0002F283D3A33344E49404752555C5B7671F6
:10730000787F6A6D64633E39303722252C2B060165
:10731000080F1A1D1413AEA9A0A7B2B5BCBB969155
:10732000989F8A8D8483DED9D0D7C2C5CCCBE6E1C5
:10733000E8EFFAFDF4F30000FFFFFFFF000000009C
:10734000672B0000FFFF00000000000000000000AD
:10735000FFFF00000000000000000000FFFF000031
:107360000000000000000000FFFF0000000000001F
:1073700000000000FFFF000000000000000000000F
:10738000FFFF00000000000000000000FFFF000001
:107390000000000000000000FFFF000000000000EF
:1073A00000000000FFFF00000000000000000000DF
:1073B000FFFF00000000000000000000FFFF0000D1
:1073C0000000000000000000FFFF000000000000BF
:1073D00000000000FFFF00000000000000000000AF
:1073E000FFFF00000000000000000000FFFF0000A1
:1073F000000000000000000080813A3B3C3D3E3030
:1074000031323334353649858683848E8F3F4053FD
:107410009192000000000000000000000000000049
:107420000000000000000000544653333632303074
:10743000000000001E001F00000006000C000B00F2
:107440000F00040007000F000300040006000A00FC
:107450000B000C003230323630313037000000087B
:107460000010002000400080FFFF7D00FA00F401C2
:10747000E803D007A00FFFFF00000000FFFF00009F
:10748000000010270000E803FFFF00000000FFFFDE
:1074900000000000FFFF00000000FFFF00000000F0
:1074A000FFFF00000000050000000100FFFF0000DA
:1074B0000000FFFF00000000FFFF00000000FFFFD2
:1074C00000000000FFFF00000000FFFF00000000C0
:1074D000FFFF00000000FFFF00000000FFFF0000B2
:1074E0000000FFFF00000000FFFF00000000FFFFA2
:1074F00000000000FFFF00000000BC340429D4306D
:10750000FFFF00000000FFFF00000000FFFF000081
:107510000000FFFF00000000FFFF00000000FFFF71
:1075200000000000FFFF00000000FFFF000000005F
:10753000010000000000FFFF00000000803E64002A
:10754000B80BFFFF00000000FFFF00000000FFFF7E
:1075500000000000FFFF00000000FFFF000000002F
:10756000FFFF00000000FFFF00000000FFFF000021
:107570000000FFFF00000000FFFF00000000FFFF11
:1075800000000000FFFF00000000FFFF00000000FF
:10759000FFFF00000000FFFF00000000FFFF0000F1
:1075A0000000FFFF00000000FFFF00000000D00708
:1075B0000A006400F82A4C1D10276842A438983A43
:1075C000FFFF00000000FFFF00000000FFFF0000C1
:1075D0000000FFFF00000000FFFF00000000FFFFB1
:1075E0000000000060EA8813008060EA88130080D1
:1075F000FFFF00000000FFFF00000000FFFF000091
:107600000000FFFF00000000FFFF0000000064001A
:1076100000001900FFFF00000000FFFF0000000055
:10762000FFFF00000000FFFF00000000FFFF000060
:107630000000800001002000640000001E00FFFF29
:1076400000000000FFFF00000000FFFF000000003E
:10765000E80301000100FFFF00000000FFFF000041
:107660000000FFFF00000000FFFF00000000FFFF20
:1076700000000000FFFF00000000FFFF000000000E
:10768000FFFF00000000A00F0000C409FFFF000082
:107690000000FFFF00000000FFFF00000000FFFFF0
:1076A00000000000FFFF00000000FFFF00000000DE
:1076B000FFFF00000000FFFF00000000FFFF0000D0
:1076C0000000FFFF00000000FFFF00000000FFFFC0
:1076D00000000000FFFF00000000FFFF00000000AE
:1076E000FFFF00000000FFFF00000000FFFF0000A0
:1076F0000000FFFF00000000FFFF00000000FFFF90
:1077000000000000FFFF00000000FFFF000000007D
:10771000FFFF000000000000000000000000002F3C
:10772000000000000700070000147F147F140024ED
:107730002A7F2A120062640813230036495522501A
:1077400000000503000000001C224100000041224F
:107750001C000014083E08140008083E0808000039
:1077600000A0600000080808080800006060000031
:10777000002010080402003E5149453E0000427FAF
:107780004000004261514946002141454B310018FB
:1077900014127F10002745454539003C4A494930BD
:1077A0000001710905030036494949360006494977
:1077B000291E000036360000000056360000000882
:1077C000142241000014141414140000412214085F
:1077D00000020151090600324959513E007C121144
:1077E000127C007F49494936003E41414122007FD9
:1077F0004141221C007F49494941007F0909090193
:10780000003E4149497A007F0808087F0000417F17
:107810004100002040413F01007F08142241007FC9
:1078200040404040007F020C027F007F0408107F30
:10783000003E4141413E007F09090906003E415199
:10784000215E007F09192946004649494931000156
:10785000017F0101003F4040403F001F2040201FAA
:10786000003F4038403F006314081463000708706D
:10787000080700615149454300007F414100005520
:107880002A552A55000041417F00000402010204EC
:1078900000404040404000000102040000205454D9
:1078A0005478007F48444438003844444420003829
:1078B0004444487F00385454541800087E0901029B
:1078C0000018A4A4A47C007F080404780000447D70
:1078D0004000004080847D00007F102844000000AC
:1078E000417F4000007C04180478007C0804047880
:1078F00000384444443800FC24242418001824246C
:1079000018FC007C08040408004854545420000467
:107910003F444020003C4040207C001C2040201C74
:10792000003C4030403C004428102844001CA0A0EB
:10793000A07C004464544C44141414141414000027
:10794000000000000000000000000000FC0000003B
:10795000000002000000000C020C02000000000009
:10796000000090D0BCD0BC9000030003000018249D
:10797000FE448C000302070201001824D8B04C809A
:10798000000300010201C038E438E00001020201F6
:1079900002020806000000000000000000000000D5
:1079A00000F80402000000010204000204F80000D4
:1079B0000004020100009060F860900000000100E7
:1079C00000002020FC20200000000100000000003A
:1079D00000000000080600000000202020202000F9
:1079E0000000000000000000000000000002000095
:1079F00000000080601C0200040300000000F80486
:107A00000404F8000102020201000008FC0000006A
:107A1000000203020000188444241800030202023A
:107A2000020008042424D80001020202010040B030
:107A300088FC80000000000302003C242424C400D1
:107A4000010202020100F824242CC00001020202FB
:107A500001000C04E41C0400000003000000D82412
:107A60002424D80001020202010038444444F800F2
:107A700000030202010000001000000000000200EC
:107A800000000000200000000000060000000020B0
:107A90005088040200000000010290909090900035
:107AA00000000000000000020488502000020100D5
:107AB00000001804C4241800000002000000F804AC
:107AC000E494F80001020202020000E09CF0800051
:107AD00002030000030204FC2424D8000203020273
:107AE0000100F80404040C0001020202010004FC7D
:107AF0000404F80002030202010004FC24740C00D8
:107B000002030202030004FC24740C0002030200BE
:107B10000000F0080444CC4000010202010004FC13
:107B20002020FC040203000003020404FC040400FF
:107B3000020203020200000404FC0404060404031D
:107B4000000004FC24D00C0402030200030204FC25
:107B500004000000020302020203FC3CC03CFC00E3
:107B600003000300030004FC30C4FC040203020011
:107B70000300F8040404F80001020202010004FCFE
:107B800024241800020302000000F8848404F80092
:107B900001020207050004FC2464980002030200AD
:107BA0000302182424448C000302020201000C0486
:107BB000FC040C0000020302000004FC0000FC04B2
:107BC000000102020100047C80E01C0400000300AC
:107BD00000001CE03CE01C00000300030000049CCB
:107BE000609C0400020300030200041CE01C04006B
:107BF0000002030200000C84641C04000203020261
:107C000003000000FE020200000007040400000E52
:107C100030C00000000000010200000202FE00006F
:107C2000000404070000000402040000000000003B
:107C30000000000000000000080808080808000014
:107C4000020000000000000000000040A0A0C000F2
:107C500000010202030204FC2020C0000003020213
:107C6000010000C02020600000010202020000C0EC
:107C70002024FC0000010202030200C0A0A0C000FA
:107C80000001020202000020F82424040002030282
:107C900002000040A0A0602000070A0A0A0404FCB9
:107CA0002020C0000203020003020020E4000000C4
:107CB000000203020000000020E40000080808079A
:107CC000000004FC80E02020020302000302040400
:107CD000FC000000020203020200E020E020C000DD
:107CE00003000300030020E02020C0000203020084
:107CF000030200C02020C00000010202010020E0B9
:107D00002020C000080F0A02010000C02020E0006F
:107D10000001020A0F0820E04020200002030200B8
:107D200000000060A0A0200000020202030000206A
:107D3000F820000000000102020020E00020E00026
:107D400000010202030220E0208060200000030105
:107D500000006080E08060000003000300002060FD
:107D60008060200002030003020020E020806020E9
:107D70000808070100000020A060200000020302A4
:107D80000200000020DE02000000000704000000E6
:107D900000FF00000000000F00000002DE200000D5
:107DA00000040700000002010204040200000000B9
:107DB00000000000000000000000000000000000C3
:107DC0000000000000F80000000000000033300058
:107DD000000000100C06100C06000000000000005F
:107DE000000040C07840C0784000043F04043F04D5
:107DF0000400007088FC08300000001820FF211EDD
:107E00000000F008F000E018000000211C031E2113
:107E10001E0000F00888700000001E21232419278E
:107E2000211010160E0000000000000000000000ED
:107E30000000000000E01804020000000007182005
:107E4000400000020418E000000000402018070075
:107E50000000404080F0804040000202010F01021B
:107E60000200000000F0000000000101011F0101FC
:107E70000100000000000000000080B07000000061
:107E800000000000000000000000000101010101ED
:107E90000101000000000000000000303000000080
:107EA0000000000000008060180400601806010057
:107EB000000000E010080810E000000F1020201063
:107EC0000F00001010F8000000000020203F2020CC
:107ED0000000007008080888700000302824222163
:107EE0003000003008888848300000182020201119
:107EF0000E000000C02010F8000000070424243FFA
:107F0000240000F8088888080800001921202011A2
:107F10000E0000E0108888180000000F11202011CA
:107F20000E0000380808C83808000000003F0000B4
:107F300000000070880808887000001C222121229F
:107F40001C0000E010080810E0000000312222119F
:107F50000F00000000C0C000000000000030300032
:107F600000000000008000000000000080600000B1
:107F700000000000804020100800000102040810EA
:107F800020004040404040404000040404040404F9
:107F900004000008102040800000002010080402A7
:107FA0000100007048080808F000000000303601A9
:107FB0000000C030C828E810E00007182724231468
:107FC0000B000000C038E0000000203C2302022724
:107FD000382008F8888888700000203F2020201171
:107FE0000E00C030080808083800071820202010AC
:107FF000080008F808080810E000203F20202010A2
:108000000F0008F88888E8081000203F202023206F
:10801000180008F88888E8081000203F20000300B6
:108020000000C03008080838000007182020221E71
:10803000020008F808000008F808203F210101218B
:108040003F20000808F8080800000020203F2020FA
:10805000000000000808F8080800C08080807F0049
:10806000000008F888C028180800203F20012638A2
:10807000200008F8080000000000203F20202020F9
:10808000300008F8F800F8F80800203F003F003FF3
:10809000200008F830C00008F808203F200007182A
:1080A0003F00E01008080810E0000F10202020100A
:1080B0000F0008F808080808F000203F210101011E
:1080C0000000E01008080810E0000F1824243850C1
:1080D0004F0008F8888888887000203F2000030C33
:1080E000302000708808080838000038202121223C
:1080F0001C00180808F8080818000000203F20009D
:10810000000008F808000008F808001F20202020C0
:108110001F000878880000C83808000007380E01E2
:108120000000F80800F80008F800033C0700073CCE
:108130000300081868808068180820302C03032C7E
:1081400030200838C800C83808000000203F200050
:10815000000010080808C838080020382621202010
:108160001800000000FE020202000000007F4040F4
:108170004000000C30C00000000000000001063884
:10818000C00000020202FE000000004040407F00EC
:1081900000000000040202020400000000000000D1
:1081A00000000000000000000000808080808080CF
:1081B00080800002020400000000000000000000B7
:1081C000000000008080808000000019242222220C
:1081D0003F2008F8008080000000003F112020119F
:1081E0000E000000008080800000000E1120202082
:1081F0001100000000808088F800000E112020107F
:108200003F200000808080800000001F2222222268
:108210001300008080F0888888180020203F2020EC
:1082200000000000808080808000006B9494949314
:10823000600008F8008080800000203F21000020BE
:108240003F2000809898000000000020203F202060
:108250000000000000809898000000C08080807FAF
:10826000000008F8000080808000203F24022D30AC
:108270002000000808F8000000000020203F202017
:1082800000008080808080808000203F20003F2090
:10829000003F8080008080800000203F210000207F
:1082A0003F200000808080800000001F20202020D0
:1082B0001F00808000808000000080FFA12020112E
:1082C0000E000000008080808000000E112020A0A1
:1082D000FF80808080008080800020203F2120005F
:1082E000010000008080808080000033242424244A
:1082F0001900008080E0808000000000001F202026
:1083000000008080000000808000001F20202010DE
:108310003F20808080000080808000010E300806B1
:10832000010080800080008080800F300C030C30C2
:108330000F0000808000808080000020312E0E31F0
:108340002000808080000080808080818E701806F0
:10835000010000808080808080000021302C22215C
:10836000300000000000807C020200000000003F9E
:10837000404000000000FF00000000000000FF007F
:1083800000000002027C800000000040403F00002E
:1083900000000006010102020404000000000000C9
:1083A00000000000000000000000000000000000CD
:1083B00000000000000000000000000000000000BD
:1083C0000000000000000000000000F0F0F00000DD
:1083D00000000000000000017F010000000000001C
:1083E0000000001C1C1C0000000000008060301C0D
:1083F0008C60301C0C000000000000000000000039
:10840000000000000000000000000000000000006C
:1084100000E00000000000E000000086E69F868685
:108420008686E69F860000011F01010101011F01F0
:108430000100000080C06020F820E0C000000000C3
:1084400003070C18FF70E18100000000070F1010F7
:108450007F100F0700008060206080000000E02097
:1084600000000F3020309F70DC371030C00000005B
:10847000100E03000718101807000000C02020E0AD
:10848000C0000000000080E01F38E88703C43C04FF
:108490000000070F1810100B070D101008000080C7
:1084A0008C4C3800000000000000000000000000BC
:1084B00000000000000000000000000000000000BC
:1084C000000000000000000080E030080400000010
:1084D000000000FEFF01000000000000000000009E
:1084E000030F1820400000040830E0800000000066
:1084F00000000000000001FFFE000000000000403E
:1085000020180F0300000000000000000000000021
:10851000C00000000000004266663C18FF183C6680
:1085200066420000000000000300000000000000A0
:10853000000000008000000000000010101010106B
:10854000FF101010101000000000000003000000D9
:10855000000000000000000000000000000000001B
:108560000000000000000000000000808C4C38007B
:1085700000000000000000000000000000000000FB
:10858000000000101010101010101010100000004B
:1085900000000000000000000000000000000000DB
:1085A00000000000000000000000000000000000CB
:1085B000000000001C1C1C00000000000000000067
:1085C000000000000000E0380C0000000000807097
:1085D0001C03000000000060380E010000000000D5
:1085E0000000000080C060202060C080000000FE0D
:1085F000FF010000000001FFFE000001070E18103F
:1086000010180E0701000000808080C0E00000000C
:1086100000000000000000FFFF000000000000005C
:108620001010101F1F10101000000080402020208C
:108630002060C080000000030300804020381F0736
:108640000000001C1A1918181818181F00000080C4
:10865000C020202060C08000000000030300101034
:10866000182FE780000000070F10101010180F07D8
:108670000000000000000000C0E0F000000000C0AA
:10868000B088868180FFFF8080000000000000101D
:10869000101F1F1010000000E060606060606060EC
:1086A000000000003F1008080818F0E00000000774
:1086B0000B101010101C0F030000000080C04020A1
:1086C0002020E0C0000000FCFF211008080818F07E
:1086D000E0000001070C18101010080F0300000044
:1086E000C0E06060606060E06000000003000000C7
:1086F000E0180700000000000000001F1F0000003D
:1087000000000080C0602020202060C08000008722
:10871000EF2C1818303068CF830000070F081010B6
:108720001010180F07000000C0C020202020C080BB
:108730000000001F3F604040402010FFFE0000008E
:108740000C1C101010080F030000000000000000B7
:1087500000000000000000000000000E0E0E0000EF
:10876000000000000000001C1C1C000000000000B5
:108770000000000000000000000000000000000CED
:108780000C0000000000000000000058380000004D
:1087900000000000000000000080402010000000E9
:1087A00010284482010000000000000000000000CA
:1087B000010204081000000000000000000000009A
:1087C0000000008484848484848484848400000081
:1087D00000000000000000000000000010204080A9
:1087E000000000000000000000000000018244289A
:1087F000100000001008040201000000000000C08A
:1088000020201010101030E0C0000003030000F022
:1088100010080C070300000000001C1C1C000000D6
:108820000000000000C0406020202040C00000FC8C
:10883000FF01F00E03C1FE03807F0001070E081147
:108840001110110904020000000080E0E0000000A7
:1088500000000000807C4340477FF8800000101833
:108860001F1000000000131F1C1020E0E02020203B
:108870002060C080000000FFFF10101010182FE7CC
:108880008000101F1F1010101010180F070000009C
:1088900080C0402020202060E00000FCFF0100009C
:1088A0000000000001000001070E1810101008045D
:1088B000030020E0E02020202040C080000000FFD6
:1088C000FF000000000001FFFE00101F1F1010102D
:1088D00018080E07010020E0E02020202020206062
:1088E000800000FFFF101010107C00000000101F1F
:1088F0001F10101010101018060020E0E02020209B
:1089000020206060800000FFFF101010107C00002D
:108910000100101F1F1000000000000000000000F8
:1089200080C06020202040E0000000FCFF0100002B
:108930004040C0C140400001070E181010100F0F3A
:10894000000020E0E0200000000020E0E02000FF28
:10895000FF101010101010FFFF00101F1F1000005C
:108960000000101F1F100000202020E0E020202029
:1089700000000000000000FFFF00000000000000F9
:108980001010101F1F101010000000000000202009
:1089900020E0E020202000000000000000FFFF0099
:1089A00000000060E0808080C07F3F00000020E089
:1089B000E020000020A06020200000FFFF30187C95
:1089C000E3C000000000101F1F10000001131F1C57
:1089D000181020E0E020000000000000000000FF70
:1089E000FF000000000000000000101F1F1010100A
:1089F00010101018060020E0E0E000000000E0E0A9
:108A0000E02000FF013FFEC0E01E01FFFF00101F3D
:108A10001000031F0300101F1F1020E0E0C0000023
:108A200000000020E02000FF0003071C78E0800029
:108A3000FF00101F100000000000030F1F000000C7
:108A400080C060202060C080000000FEFF010000A8
:108A5000000000FFFE000001070E181010180C07A0
:108A6000010020E0E0202020202060C0800000FFE6
:108A7000FF2020202020301F0F00101F1F1000009B
:108A8000000000000000000080C060202060C08066
:108A9000000000FEFF010000000000FFFE000001DA
:108AA000070E1111133C7C67210020E0E0202020FC
:108AB000202060C0800000FFFF101030F0D0080FB1
:108AC0000700101F1F10000000030F1C1010008073
:108AD000C060202020204040E00000070F0C181844
:108AE000303060E08100001F0C0810101010180FCB
:108AF00007008060202020E0E0202020608001002E
:108B0000000000FFFF000000000100000000101F37
:108B10001F100000000020E0E02000000000002006
:108B2000E02000FFFF00000000000000FF00000741
:108B30000F1810101010100807002060E0E020004F
:108B4000000020E060200000077FF88000807C03A8
:108B5000000000000000071F1C070000000020E0CC
:108B6000E02000E0E0200020E0200007FFF8E01F08
:108B7000FFFCE01F00000000031F0300011F0300B3
:108B80000000002060E0A0000020E0602000000065
:108B900000038F7CF8C6010000000010181E1300AF
:108BA00001171F1810002060E0E02000000020E006
:108BB0006020000001073EF8E018070000000000F8
:108BC0000010101F1F1010000000008060202020E7
:108BD00020A0E0E0200000000000C0F03E0F0300F5
:108BE000000000101C1F17101010101806000000C5
:108BF000000000FC0404040404000000000000FF66
:108C000000000000000000000000007F40404040E5
:108C10004000000010E00000000000000000000024
:108C20000000031C60800000000000000000000045
:108C300000030C70800000000404040404FC000025
:108C4000000000000000000000FF00000000000025
:108C500040404040407F0000000000000010080C31
:108C6000040C0810000000000000000000000000DC
:108C700000000000000000000000000000000000F4
:108C800000000000000000000000000000000000E4
:108C900000000000000080808080808080808080D4
:108CA00080800000000404080800000000000000AC
:108CB00000000000000000000000000000000000B4
:108CC00000000000000000000000000000000000A4
:108CD0000000000098D844642424FCF80000000F31
:108CE0001F18101010081F1F10180020E0F00000BF
:108CF0000000000000000000FFFF180804040CF84A
:108D0000F00000001F0F18101010180F03000000D3
:108D10000000000000000000000000E0F81804045B
:108D2000043C3800000000030F0C1010101008065F
:108D300000000000000000000020E0F0000000E063
:108D4000F81C04040408FFFF000000030F181010B3
:108D500010081F0F080000000000000000000000C5
:108D600000000000E0F8484444444C7870000000E3
:108D7000030F0C181010100804000000000080C041
:108D8000602020E0C00000040404FFFF0404040489
:108D90000000000010101F1F101010000000000045
:108DA00000000000000000000000000070F88C04CB
:108DB000048CF874040C007076CF8D8D8D89C87882
:108DC00070000020E0F00000000000000000000043
:108DD000FFFF08040404FCF8000000101F1F10002F
:108DE00000101F1F10000000000000606000000065
:108DF00000000000040404FCFC000000000000006F
:108E00001010101F1F1010100000000000000000C4
:108E100000606000000000000000040404FCFC008E
:108E200000000000C0C08080C07F3F000000002024
:108E3000E0F000000000000000000000FFFF80C024
:108E4000F41C0404000000101F1F1100031F1C105D
:108E500010000000202020E0F000000000000000D2
:108E6000000000FFFF000000000000001010101FB5
:108E70001F101010000000000000000000000000A3
:108E8000000004FCFC0804FCFC0804FCFC00101FAF
:108E90001F10001F1F10001F1F1000000000000007
:108EA0000000000000000004FCFC08080404FCF8BA
:108EB000000000101F1F100000101F1F10000000F6
:108EC0000000000000000000000000E0F0180C04AA
:108ED000040C18F0E00000030F0C101010100C0F21
:108EE000030000000000000000000000000000047B
:108EF000FCFC080404040CF8F0000080FFFF8890DC
:108F000010101C0F03000000000000000000000013
:108F1000000000E0F81C04040408F8FC0000000352
:108F20000F1810109088FFFF800000000000000064
:108F3000000000000000040404FCFC100804040C01
:108F40000C001010101F1F10101000000000000077
:108F50000000000000000000000000003078CCC4D9
:108F60008484840C1C0000001E1810101011190FAE
:108F700006000000000000C0000000000000000427
:108F80000404FFFF040404000000000000000F1FA1
:108F90001010100C00000000000000000000000095
:108FA00000000004FCFE00000004FCFE00000000C5
:108FB0000F1F181010081F0F08000000000000000D
:108FC00000000000000000040C3CFCC40000C43C95
:108FD0000C0400000000010F1E0E01000000000044
:108FE00000000000000000000000043CFCC400E49D
:108FF0007CFC84807C040000071F070000071F071B
:10900000000000000000000000000000000000045C
:10901000041C7CE4C0341C0404000010101C160165
:10902000131F1C18100000000000000000000000CA
:10903000000000040C3CFCC400C43C04040000001C
:10904000C080C1370E0100000000000000000000D9
:1090500000000000000000001C0404C4F47C1C0498
:1090600000000000101C1F17111010180E00000047
:109070000000000000F80C040000000000000010D8
:1090800028EF00000000000000000000003F6040EA
:109090000000000000000000FF00000000000000D1
:1090A00000000000FF0000000000000000000000C1
:1090B000FF00000000000000040CF80000000000A9
:1090C000000000000000EF28100000000000000079
:1090D00040603F000000000000000018060202048B
:1090E00008102020300800000000000000000000F0
:1090F0000000000000000000000000000000000070
:10910000C012000080250000004B00000096000007
:1091100000E1000000C201000000000040910008D2
:1091200000000020200000008E6D00086091000803
:1091300020000020C81D00009E6D000800000000F7
:1091400002000102030405060708090A0B000000DB
:109150000024F400010000000000000000000000F6
:04000005080000C12E
:00000001FF
